:020000020000FC
:100000000C94D32E18951895189518951895189541
:100010001895189518951895189518951895189578
:100020001895189518951895189518951895189568
:100030001895189518951895189518951895189558
:100040001895189518951895189518951895189548
:100050000C94A40B18951895189518951895189543
:100060001895189518951895189518951895189528
:100070001895189518951895189518951895189518
:100080001895189518951895189518951895189508
:1000900018951895189518951895189518951895F8
:1000A00018951895189518951895189518951895E8
:1000B00018951895189518951895189518951895D8
:1000C00018951895189518951895189518951895C8
:1000D00018951895189518951895189518951895B8
:1000E00018951895189518951895189518951895A8
:1000F0001895189518951895189518951895189598
:100100001895189518951895189518951895189587
:100110001895189518951895189518950C94930B93
:100120001895189518951895189518951895189567
:10013000189518950C94150B1895189518951895F1
:100140001895189518951895189518951895189547
:100150001895189518951895189518951895189537
:100160001895189518951895189518951895189527
:100170001895189518951895189518951895189517
:100180001895189518951895189518951895189507
:1001900018951895189518951895189518951895F7
:1001A00018951895189518951895189518951895E7
:1001B00018951895189518951895189518951895D7
:1001C00018951895189518951895189518951895C7
:1001D00018951895189518951895189518951895B7
:1001E00018951895189518951895189518951895A7
:1001F00018951895189518951895189544241FBCAE
:1002000037CB7ABC26B8A2BD41F61CBE6EBA0DBE75
:10021000FC0C633C5C1D633E6EE3A33E5C1D633ED1
:10022000FC0C633C6EBA0DBE41F61CBE26B8A2BDE6
:1002300037CB7ABC44241FBC21C181BAC40C6C3AB0
:10024000EEC16F3BD2AB8C3BC90CE4BA005798BCF3
:10025000A99942BD8017AEBDDA0CFCBDC63C1BBEE1
:10026000B8DB563FC63C1BBEDA0CFCBD8017AEBDEA
:10027000A99942BD005798BCC90CE4BAD2AB8C3BDB
:10028000EEC16F3BC40C6C3A21C181BA14BEA1BD52
:100290006FEDFCBDDC252FBEE9383F3FDC252FBECE
:1002A0006FEDFCBD14BEA1BDE5FF3CBE6A8B31BE47
:1002B000D6704CBC0186593E0595A33E0186593E39
:1002C000D6704CBC6A8B31BEE5FF3CBE6B55E8BCBA
:1002D000DF5B27BE8B692EBE0921243EE2D3CE3ED2
:1002E0000921243E8B692EBEDF5B27BE6B55E8BC1F
:1002F0007F0161B9FBB310BB8A3F00BCBCDAADBC67
:1003000045BC4ABDA7EBD2BD597F45BEAC84403F3A
:10031000597F45BEA7EBD2BD45BC4ABDBCDAADBCDA
:100320008A3F00BCFBB310BB7F0161B91F1F1F00D8
:10033000000000001C1E1F1F1F1F1F1F1F1F1F1F4D
:100340001F1F1E1C00000000001F1F1F1F1F1F1F5C
:100350001F1F0F07070F1F1F1F1F1F1F0000000079
:10036000001F1F1F1F1F1F00001F1F1F050001046C
:1003700003022020052020FF0007010403060007D8
:10038000010603020506FF2020FF05070006030201
:100390000507000403020000012020FF05070104F7
:1003A00003020507010303020507070420200507D0
:1003B00007040303050701042020001F2C406300ED
:1003C0000102040810204024212A21302136213D39
:1003D000214121442148214D21522157212A2A2AF5
:1003E0002A2A2A2A2A2A0000AF2510003620E421D2
:1003F0003E228622B822FD222D235D23A023032442
:100400003C247524AF24EF24352573250000122CDD
:100410001000052A442A572A6C2A8B2AB62AE12A78
:10042000082B192B2A2B3B2B522B6C2B812BF42BBB
:10043000052C0000222E1000282C6C2C7F2C942CD4
:10044000AD2CD82C012D262D372D482D592D702D52
:100450008A2D9F2D042E152E0001A0349D34459029
:100460003402903411FA330BBF3301183401903445
:1004700001903401903402183405AC3301ED33019E
:10048000FA3303C83302FA3303F633FB03E330D005
:1004900000EC1BE237D100EC1BE234D100EC1BE294
:1004A00031D103E325D000EC1BE22CD103E320D0B3
:1004B00000E614E027D102E01BD000E614E022D1D0
:1004C00008E016D000E614E01DD101E011D000ECE8
:1004D0001BE218D100EC1BE215D106E009D000E6C2
:1004E00014E010D10CE004D000E614E00BD1089524
:1004F0008A93802FE4E4F6E000810F7B008308E319
:1005000010E000D100916406007F00936406082F7C
:1005100002950F7010916406102B10936406E4E4AA
:10052000F6E000810068008308E310E0EBD0E4E42B
:10053000F6E000810F77008308E111E0E3D000913D
:100540006406007F009364068F7000916406082B98
:1005500000936406E4E4F6E000810068008308E3A9
:1005600010E0D0D0E4E4F6E000810F77008308E1EA
:1005700011E0C8D0899108958A93802FE4E4F6E0D1
:1005800000810064008308E310E0BCD000916406A1
:10059000007F00936406082F02950F701091640687
:1005A000102B10936406E4E4F6E0008100680083F9
:1005B00008E310E0A7D0E4E4F6E000810F770083C1
:1005C00008E111E09FD000916406007F009364066B
:1005D0008F7000916406082B00936406E4E4F6E053
:1005E00000810068008308E310E08CD0E4E4F6E0CA
:1005F00000810F77008308E111E084D0899108958C
:100600000E945832C801A0E007C0B0E0FC01EA0F28
:10061000FB1F0081B1DFA395B0E0FC01EA0FFB1FD7
:100620000081002311F0A13180F3E4E00C946932E1
:100630005FDF0FE915E2E4DF08951BEC1093520031
:1006400018E010935000E1E5F0E0108113FFFBCFBC
:10065000003221F402EC0093550003C003EC009338
:100660005500E0E5F0E0008100610083E1E5F0E0A5
:10067000008104FFFBCF08ED04BF04E000934000BD
:10068000E0E5F0E000810E7F0083089504E414E0CB
:1006900000930C0210930D0200E10093010202E2AC
:1006A0000093020203E00093040203E0009320029F
:1006B00008E200932102E0E0F2E0008101600083A3
:1006C000089501E00093280200E3009329020895B1
:1006D00001E00093300208E30093310208950DE039
:1006E0000093200300E40093210300E00093220321
:1006F00000E50093240300E70093280300EE009335
:100700002A0308950150104098018901232BD1F745
:1007100008958A93802F04C008EE1DEF0E94651093
:100720008A95082F802F0023B9F7899108950E9498
:10073000573280E090E0A0E0B0E04EE0442E1BC0D5
:10074000442D50E0440F551F440F551FFA01E55545
:10075000FA4D0080118022803380442D50E0440FF8
:10076000551F440F551FFA01E155FA4D00821182C1
:10077000228233824A9441E0441610F7EFEAF5E210
:100780000083118322833383442423C0042D10E08B
:10079000000F111F000F111FF801E450FE4F45918B
:1007A000559165917491042D10E0000F111F000FF9
:1007B000111FF801E155FA4D008111812281338129
:1007C0000E94DC30AC01BD010E947B30C801D90120
:1007D00043940FE04016D0F28C019D01E5E00C94AB
:1007E00068320E94573280E090E0A0E0B0E04EE036
:1007F000442E1BC0442D50E0440F551F440F551F7D
:10080000FA01E951FA4D0080118022803380442D95
:1008100050E0440F551F440F551FFA01E551FA4DA2
:1008200000821182228233824A9441E0441610F7FA
:10083000EBEEF5E20083118322833383442423C04B
:10084000042D10E0000F111F000F111FF801E450DC
:10085000FE4F4591559165917491042D10E0000F64
:10086000111F000F111FF801E551FA4D0081118190
:10087000228133810E94DC30AC01BD010E947B30BB
:10088000C801D90143940FE04016D0F28C019D01BC
:10089000E5E00C9468320E94573280E090E0A0E0DE
:1008A000B0E04EE0442E1BC0442D50E0440F551FD5
:1008B000440F551FFA01ED5DF94D00801180228033
:1008C0003380442D50E0440F551F440F551FFA014B
:1008D000E95DF94D00821182228233824A9441E01F
:1008E000441610F7E7E2F6E2008311832283338394
:1008F000442423C0042D10E0000F111F000F111F0E
:10090000F801E450FE4F4591559165917491042D85
:1009100010E0000F111F000F111FF801E95DF94DE4
:1009200000811181228133810E94DC30AC01BD0144
:100930000E947B30C801D90143940FE04016D0F2E9
:100940008C019D01E5E00C9468320E94573280E0F2
:1009500090E0A0E0B0E044E1442E1BC0442D50E004
:10096000440F551F440F551FFA01E15AF94D0080FD
:10097000118022803380442D50E0440F551F440FD6
:10098000551FFA01ED59F94D0082118222823382FE
:100990004A9441E0441610F7E3E6F6E2008311833F
:1009A00022833383442423C0042D10E0000F111F41
:1009B000000F111FF801E85CFD4F459155916591BD
:1009C0007491042D10E0000F111F000F111FF8018A
:1009D000ED59F94D00811181228133810E94DC3073
:1009E000AC01BD010E947B30C801D901439405E1EF
:1009F0004016D0F28C019D01E5E00C9468320E9413
:100A0000573280E090E0A0E0B0E044E1442E1BC00B
:100A1000442D50E0440F551F440F551FFA01ED546B
:100A2000F94D0080118022803380442D50E0440F26
:100A3000551F440F551FFA01E954F94D00821182E8
:100A4000228233824A9441E0441610F7E7EBF6E243
:100A50000083118322833383442423C0042D10E0B8
:100A6000000F111F000F111FF801E85CFD4F4591A9
:100A7000559165917491042D10E0000F111F000F26
:100A8000111FF801E954F94D008111812281338150
:100A90000E94DC30AC01BD010E947B30C801D9014D
:100AA000439405E14016D0F28C019D01E5E00C94E1
:100AB00068320E94573280E090E0A0E0B0E044E16C
:100AC000442E1BC0442D50E0440F551F440F551FAA
:100AD000FA01E95FF84D0080118022803380442DB7
:100AE00050E0440F551F440F551FFA01E55FF84DC4
:100AF00000821182228233824A9441E0441610F728
:100B0000EBE0F7E20083118322833383442423C084
:100B1000042D10E0000F111F000F111FF801E85CF9
:100B2000FD4F4591559165917491042D10E0000F92
:100B3000111F000F111FF801E55FF84D00811181B1
:100B4000228133810E94DC30AC01BD010E947B30E8
:100B5000C801D901439405E14016D0F28C019D01F2
:100B6000E5E00C9468320E94573280E090E0A0E00B
:100B7000B0E046E0442E1BC0442D50E0440F551F0A
:100B8000440F551FFA01E55AF84D0080118022806C
:100B90003380442D50E0440F551F440F551FFA0178
:100BA000E15AF84D00821182228233824A9441E058
:100BB000441610F7EFE5F7E20083118322833383B5
:100BC000442423C0042D10E0000F111F000F111F3B
:100BD000F801E457FD4F4591559165917491042DAD
:100BE00010E0000F111F000F111FF801E15AF84D1E
:100BF00000811181228133810E94DC30AC01BD0172
:100C00000E947B30C801D901439407E04016D0F21E
:100C10008C019D01E5E00C9468320E94573280E01F
:100C200090E0A0E0B0E046E0442E1BC0442D50E030
:100C3000440F551F440F551FFA01E958F84D008025
:100C4000118022803380442D50E0440F551F440F03
:100C5000551FFA01E558F84D008211822282338235
:100C60004A9441E0441610F7EBE7F7E20083118362
:100C700022833383442423C0042D10E0000F111F6E
:100C8000000F111FF801E457FD4F459155916591F3
:100C90007491042D10E0000F111F000F111FF801B7
:100CA000E558F84D00811181228133810E94DC30AA
:100CB000AC01BD010E947B30C801D901439407E01B
:100CC0004016D0F28C019D01E5E00C9468320E9440
:100CD000573280E090E0A0E0B0E046E0442E1BC038
:100CE000442D50E0440F551F440F551FFA01ED5697
:100CF000F84D0080118022803380442D50E0440F55
:100D0000551F440F551FFA01E956F84D0082118214
:100D1000228233824A9441E0441610F7E7E9F7E271
:100D20000083118322833383442423C0042D10E0E5
:100D3000000F111F000F111FF801E457FD4F4591DF
:100D4000559165917491042D10E0000F111F000F53
:100D5000111FF801E956F84D00811181228133817C
:100D60000E94DC30AC01BD010E947B30C801D9017A
:100D7000439407E04016D0F28C019D01E5E00C940D
:100D800068320E945432842FA52F0E941C30482FB5
:100D900050E0440F551F440F551FFA01ED54F84D14
:100DA00040815181628173810E94BF3028013901E5
:100DB0000A2F10E020E030E00E942730A801B9019E
:100DC000820193010E945531482F50E0440F551F76
:100DD000440F551FFA01ED54F84D40815181628155
:100DE00073810E947B3090E0880F991F880F991FB4
:100DF000FC01ED54F84D0083118322833383E8E036
:100E00000C9465320E94573280E090E0A0E0B0E0A0
:100E100048E0442E1BC0442D50E0440F551F440FA2
:100E2000551FFA01E153F84D008011802280338074
:100E3000442D50E0440F551F440F551FFA01ED5249
:100E4000F84D00821182228233824A9441E0441696
:100E500010F7E3EDF7E20083118322833383442408
:100E600023C0042D10E0000F111F000F111FF80107
:100E7000E855FD4F4591559165917491042D10E011
:100E8000000F111F000F111FF801ED52F84D0081E6
:100E90001181228133810E94DC30AC01BD010E94AE
:100EA0007B30C801D901439409E04016D0F28C018F
:100EB0009D01E5E00C9468320E94573280E090E09A
:100EC000A0E0B0E048E0442E1BC0442D50E0440FA9
:100ED000551F440F551FFA01ED50F84D0080118049
:100EE00022803380442D50E0440F551F440F551F7E
:100EF000FA01E950F84D00821182228233824A942D
:100F000041E0441610F7E7EFF7E2008311832283F4
:100F10003383442423C0042D10E0000F111F000F61
:100F2000111FF801E855FD4F459155916591749158
:100F3000042D10E0000F111F000F111FF801E950E0
:100F4000F84D00811181228133810E94DC30AC0197
:100F5000BD010E947B30C801D901439409E04016CD
:100F6000D0F28C019D01E5E00C9468320E9457326A
:100F700080E090E0A0E0B0E048E0442E1BC0442DAB
:100F800050E0440F551F440F551FFA01E95EF74D1D
:100F90000080118022803380442D50E0440F551F83
:100FA000440F551FFA01E55EF74D0082118222823F
:100FB00033824A9441E0441610F7EBE1F8E20083F3
:100FC000118322833383442423C0042D10E0000FB7
:100FD000111F000F111FF801E855FD4F4591559164
:100FE00065917491042D10E0000F111F000F111F67
:100FF000F801E55EF74D00811181228133810E9465
:10100000DC30AC01BD010E947B30C801D9014394A2
:1010100009E04016D0F28C019D01E5E00C946832A5
:101020000E94573280E090E0A0E0B0E048E0442E1B
:101030001BC0442D50E0440F551F440F551FFA01AB
:10104000E55CF74D0080118022803380442D50E014
:10105000440F551F440F551FFA01E15CF74D008204
:101060001182228233824A9441E0441610F7EFE362
:10107000F8E20083118322833383442423C0042DA8
:1010800010E0000F111F000F111FF801E453FD4F76
:101090004591559165917491042D10E0000F111F39
:1010A000000F111FF801E15CF74D008111812281D1
:1010B00033810E94DC30AC01BD010E947B30C8014D
:1010C000D901439409E04016D0F28C019D01E5E07E
:1010D0000C9468320E94573280E090E0A0E0B0E0CB
:1010E00048E0442E1BC0442D50E0440F551F440FD0
:1010F000551FFA01E15AF74D00801180228033809C
:10110000442D50E0440F551F440F551FFA01ED596F
:10111000F74D00821182228233824A9441E04416C4
:1011200010F7E3E6F8E2008311832283338344243B
:1011300023C0042D10E0000F111F000F111FF80134
:10114000E453FD4F4591559165917491042D10E044
:10115000000F111F000F111FF801ED59F74D00810D
:101160001181228133810E94DC30AC01BD010E94DB
:101170007B30C801D901439409E04016D0F28C01BC
:101180009D01E5E00C9468320E94573280E090E0C7
:10119000A0E0B0E048E0442E1BC0442D50E0440FD6
:1011A000551F440F551FFA01ED57F74D0080118070
:1011B00022803380442D50E0440F551F440F551FAB
:1011C000FA01E957F74D00821182228233824A9454
:1011D00041E0441610F7E7E8F8E200831183228328
:1011E0003383442423C0042D10E0000F111F000F8F
:1011F000111FF801E453FD4F45915591659174918C
:10120000042D10E0000F111F000F111FF801E95706
:10121000F74D00811181228133810E94DC30AC01C5
:10122000BD010E947B30C801D901439409E04016FA
:10123000D0F28C019D01E5E00C9468320E94573297
:1012400080E090E0A0E0B0E04EE0442E1BC0442DD2
:1012500050E0440F551F440F551FFA01E955F74D53
:101260000080118022803380442D50E0440F551FB0
:10127000440F551FFA01E555F74D00821182228275
:1012800033824A9441E0441610F7EBEAF8E2008317
:10129000118322833383442423C0042D10E0000FE4
:1012A000111F000F111FF801E051FD4F459155919D
:1012B00065917491042D10E0000F111F000F111F94
:1012C000F801E555F74D00811181228133810E949B
:1012D000DC30AC01BD010E947B30C801D9014394D0
:1012E0000FE04016D0F28C019D01E5E00C946832CD
:1012F0000E94573280E090E0A0E0B0E04EE0442E43
:101300001BC0442D50E0440F551F440F551FFA01D8
:10131000ED51F74D0080118022803380442D50E044
:10132000440F551F440F551FFA01E951F74D008234
:101330001182228233824A9441E0441610F7E7EE8C
:10134000F8E20083118322833383442423C0042DD5
:1013500010E0000F111F000F111FF801E051FD4FA9
:101360004591559165917491042D10E0000F111F66
:10137000000F111FF801E951F74D00811181228101
:1013800033810E94DC30AC01BD010E947B30C8017A
:10139000D90143940FE04016D0F28C019D01E5E0A5
:1013A0000C9468320E94573280E090E0A0E0B0E0F8
:1013B0004EE0442E1BC0442D50E0440F551F440FF7
:1013C000551FFA01E15EF64D0080118022803380C6
:1013D000442D50E0440F551F440F551FFA01ED5D99
:1013E000F64D00821182228233824A9441E04416F3
:1013F00010F7E3E2F9E2008311832283338344246C
:1014000023C0042D10E0000F111F000F111FF80161
:10141000E051FD4F4591559165917491042D10E077
:10142000000F111F000F111FF801ED5DF64D008137
:101430001181228133810E94DC30AC01BD010E9408
:101440007B30C801D90143940FE04016D0F28C01E3
:101450009D01E5E00C9468321091480001E0009392
:1014600048002091A0003091A2000091A2000C7FC2
:1014700004600093A2004FB77894E8E4F0E00081A4
:10148000016000835091CD01EF93FF930F932F9351
:10149000EBECF1E008ED21E004BF20832F910F91E8
:1014A000FF91EF9103E00093CD01889510934800E0
:1014B0002093A0003093A2005093CD014FBF089518
:1014C000EFECF1E0008107FDFBCF0895F9DFEFECD1
:1014D000F1E0008101FF11C006E30093CA01EF9320
:1014E000FF930F932F93EBECF1E008ED21E004BFA5
:1014F00020832F910F91FF91EF9108959A938A93F2
:10150000C801DEDFFC01E05CF140F09750F440914F
:10151000EF2A50E009E010E00E94212F800F911F78
:1015200017C0803C01E0900798F44091EE2A50E00B
:1015300005E110E00E94212F98014091EF2A50E030
:101540000FE310E00E94212F200F311F820F931F05
:10155000082F0093C001892F8F718093C10100E093
:101560000093C20106E00093CA01EF93FF930F932B
:101570002F93EBECF1E008ED21E004BF20832F91E5
:101580000F91FF91EF910091C40189919991089574
:101590000E945932C801A22F00E00093060900E022
:1015A00000934608FC01E05CF140F09750F4409154
:1015B000EF2A50E009E010E00E94212F800F911FD8
:1015C00017C0803C01E0900798F44091EE2A50E06B
:1015D00005E110E00E94212F98014091EF2A50E090
:1015E0000FE310E00E94212F200F311F820F931F65
:1015F0006DDF03E30093CA01082F0093C001892F18
:101600008F718093C10100E00093C201A093C401D7
:1016100005E30093CA0120DF03E00093060901E01F
:1016200000934608E3E00C946A329A938A93FA9303
:10163000EA930A927A936A935A934A933A932A9333
:101640001A930A930FB6E0E0F2E000810460008391
:101650000091C02A10E0000F111FF801E159F64D6A
:101660000081118100933A0310933B030091C02A3B
:1016700010E0000F111FF801E15AF64D00811181B1
:1016800000933803109339030091C02A0395077023
:101690000093C02A0091C32A0023B1F100911F2AB0
:1016A0001091202A212F220F220B322F4091C02A85
:1016B00050E0440F551F440F551FFA01E152F64DFB
:1016C0004081518162817381400F511F621F731FDE
:1016D000408351836283738380912F2A9091302AB3
:1016E000019680932F2A9093302A0091312A1091ED
:1016F000322A8017910741F400E00093C32A10E0DA
:1017000000932F2A1093302A0FBE09911991299125
:10171000399149915991699179910990E991F9919A
:101720008991999118952A931A930A932FB700914A
:1017300010021091110200931F2A1093202A2FBF2C
:1017400009911991299118955A924A92BA93AA939C
:101750009A938A93FA93EA933A922A921A920A9265
:101760007A936A935A934A933A932A931A930A93D1
:101770005FB60091C32A002309F091C40091D02ADA
:101780000E5F0093DE2A80E037C05091DE2A482F9A
:10179000642F082F10E0000F111F000F111FF80118
:1017A000E152F64D008111812281338142E00E9495
:1017B0008F2F462FE6DA0E942930482F50E0440F41
:1017C000551F440F551FFA01E150F64D0083118358
:1017D0002283338300E010E020E030E0482F50E027
:1017E000440F551F440F551FFA01E152F64D008377
:1017F0001183228333838395883038F20FEF00936F
:10180000C32A00E010E020E030E0E3E4FAE20083E5
:10181000118322833383EFE3FAE20083118322836F
:101820003383EBE3FAE2008311832283338300E006
:1018300010E020E030E0EAEEFAE200831183228338
:1018400033834424C9C0042D10E0000F111F000F82
:10185000111FF801E150F64D408151816281738181
:10186000042D10E0000F111F000F111FF801E150AF
:10187000F64D00811181228133810E94672F0E94E1
:101880001C30EAEEFAE240815181628173810E944C
:101890007B30EAEEFAE20083118322833383EBE3A9
:1018A000FAE200811181228133810E941C30C8013B
:1018B000D901042D10E0000F111F000F111FF801B6
:1018C000E150F64D00811181228133810E941C304C
:1018D000442D50E0440F551F440F551FFA01E158A5
:1018E000F64D40815181628173810E94DC30AC01F0
:1018F000BD010E947B300E942930EBE3FAE20083B5
:10190000118322833383EFE3FAE200811181228184
:1019100033810E941C30C801D901042D10E0000F52
:10192000111F000F111FF801E150F64D00811181C8
:10193000228133810E941C30442D50E0440F551FFA
:10194000440F551FFA01E156F64D408151816281E5
:1019500073810E94DC30AC01BD010E947B300E948B
:101960002930EFE3FAE20083118322833383E3E437
:10197000FAE200811181228133810E941C30C8016A
:10198000D901042D10E0000F111F000F111FF801E5
:10199000E150F64D00811181228133810E941C307B
:1019A000442D50E0440F551F440F551FFA01E154D8
:1019B000F64D40815181628173810E94DC30AC011F
:1019C000BD010E947B300E942930E3E4FAE20083EB
:1019D000118322833383439408E0401608F433CF05
:1019E00040E050E060E071E4EAEEFAE2008111814B
:1019F000228133810E9455310E94C036EAEEFAE21C
:101A000000831183228333830091E22A013099F409
:101A1000EAEEFAE200811181228133810E942930AD
:101A20004091352A5091362A0E943B2F0093B42AC8
:101A30001093B52A14C0EAEEFAE2008111812281E6
:101A400033810E9429304091352A5091362A440F23
:101A5000551F0E943B2F0093B42A1093B52A009182
:101A6000DF2A10E0F801E154FC4F449150E000916E
:101A7000B42A1091B52A0E94532F0093B42A1093D0
:101A8000B52AEBE3FAE20081118122813381EFE490
:101A9000FAE20083118322833383EFE3FAE20081C9
:101AA000118122813381E3E5FAE2008311832283ED
:101AB0003383E3E4FAE20081118122813381EBE593
:101AC000FAE200831183228333830091C22A002328
:101AD00079F100E00093C22AEFE4FAE2008111817B
:101AE00022813381E3E6FAE2008311832283338388
:101AF000E3E5FAE20081118122813381EFE5FAE228
:101B00000083118322833383EBE5FAE200811181A4
:101B100022813381E7E6FAE2008311832283338353
:101B20000091B42A1091B52A0093BE2A1093BF2ABF
:101B3000E3E6FAE20081118122813381EFE4FAE2E7
:101B40004081518162817381401B510B620B730B89
:101B50004083518362837383EFE5FAE20081118150
:101B600022813381E3E5FAE2408151816281738110
:101B7000401B510B620B730B408351836283738351
:101B8000E7E6FAE20081118122813381EBE5FAE296
:101B90004081518162817381401B510B620B730B39
:101BA00040835183628373830091392A10913A2ACA
:101BB000013020E0120709F057C10091E22A0230FB
:101BC00009F4ADC00091DC2A0130B9F5EFE4FAE286
:101BD00000811181228133810E941C300E94970371
:101BE0000E942930E7E8FAE20083118322833383DD
:101BF000E3E5FAE200811181228133810E941C30E9
:101C00000E94F1030E942930EBE8FAE2008311837D
:101C100022833383EBE5FAE2008111812281338153
:101C20000E941C300E944B040E942930E3E8FAE233
:101C300000831183228333833BC10091DC2A02306D
:101C4000B9F5EFE4FAE200811181228133810E942B
:101C50001C300E94A5040E942930E7E8FAE20083C4
:101C6000118322833383E3E5FAE20081118122812B
:101C700033810E941C300E94FF040E942930EBE84F
:101C8000FAE20083118322833383EBE5FAE20081D9
:101C90001181228133810E941C300E9459050E94CB
:101CA0002930E3E8FAE2008311832283338300C101
:101CB000EFE4FAE200811181228133810E941C301D
:101CC0000E94B3050E942930E7E8FAE200831183FD
:101CD00022833383E3E5FAE200811181228133819B
:101CE0000E941C300E940D060E942930EBE8FAE2A7
:101CF0000083118322833383EBE5FAE200811181B3
:101D0000228133810E941C300E9467060E94293084
:101D1000E3E8FAE20083118322833383C9C0009190
:101D2000DC2A0130A9F5EFE4FAE200811181228179
:101D300033810E941C300E9402070E942930E7E88C
:101D4000FAE20083118322833383E3E5FAE2008120
:101D50001181228133810E941C30AED80E9429302B
:101D6000EBE8FAE20083118322833383EBE5FAE2A6
:101D700000811181228133810E941C30F7D80E949A
:101D80002930E3E8FAE2008311832283338390C091
:101D90000091DC2A0230A1F5EFE4FAE20081118122
:101DA000228133810E941C303BD90E942930E7E810
:101DB000FAE20083118322833383E3E5FAE20081B0
:101DC0001181228133810E941C3084D90E942930E4
:101DD000EBE8FAE20083118322833383EBE5FAE236
:101DE00000811181228133810E941C30CDD90E9453
:101DF0002930E3E8FAE2008311832283338358C059
:101E0000EFE4FAE200811181228133810E941C30CB
:101E100015DA0E942930E7E8FAE200831183228371
:101E20003383E3E5FAE200811181228133810E944C
:101E30001C305EDA0E942930EBE8FAE2008311835D
:101E400022833383EBE5FAE2008111812281338121
:101E50000E941C30A7DA0E942930E3E8FAE20083EE
:101E600011832283338324C0EFE4FAE200811181DD
:101E700022813381E7E8FAE20083118322833383EE
:101E8000E3E5FAE20081118122813381EBE8FAE295
:101E90000083118322833383EBE5FAE20081118111
:101EA00022813381E3E8FAE20083118322833383C2
:101EB0000091D72A00950093D72A0091D72A0023B2
:101EC00009F0C9C0E7E8FAE200811181228133817B
:101ED000E3E9FAE24081518162817381040F151FA9
:101EE000261F371FEFE9FAE2008311832283338331
:101EF000EBE8FAE20081118122813381E7E9FAE21D
:101F00004081518162817381040F151F261F371F85
:101F1000E3EAFAE20083118322833383E3E8FAE2FF
:101F20000081118122813381EFE8FAE24081518101
:101F300062817381040F151F261F371FEBE9FAE238
:101F400000831183228333830091D82A0095009364
:101F5000D82A0091D82A002309F058C0EFE9FAE204
:101F60000081118122813381E7EAFAE240815181C7
:101F700062817381040F151F261F371F42E050E056
:101F800060E070E00E94BA2FE7E4FAE20083118378
:101F900022833383E3EAFAE20081118122813381D3
:101FA000EBEAFAE24081518162817381040F151FCF
:101FB000261F371F42E050E060E070E00E94BA2F19
:101FC000EBE4FAE20083118322833383EBE9FAE244
:101FD0000081118122813381EFEAFAE2408151814F
:101FE00062817381040F151F261F371F42E050E0E6
:101FF00060E070E00E94BA2FE7E5FAE20083118307
:10200000228333830FEF0093D92A49C0EFE9FAE224
:102010000081118122813381E7EAFAE20083118392
:1020200022833383E3EAFAE2008111812281338142
:10203000EBEAFAE20083118322833383EBE9FAE2CD
:102040000081118122813381EFEAFAE2008311835A
:102050002283338324C0E7E8FAE2008111812281E0
:102060003381E3E9FAE20083118322833383EBE8CF
:10207000FAE20081118122813381E7E9FAE20083EB
:10208000118322833383E3E8FAE200811181228104
:102090003381EFE8FAE200831183228333835FBE4A
:1020A00009911991299139914991599169917991A0
:1020B0000990199029903990E991F9918991999114
:1020C000A991B9914990599018959C01C80101971F
:1020D000FC01CF01EF2BD9F716950795C8010197A1
:1020E000FC01CF01EF2BD9F7C90108950E945832A6
:1020F00000E40E947802AFEF80E002C0A6958395CD
:102100008830A8F4BA2F90E005C000E00E94BC021D
:10211000B6959395983090F7BB2311F001E001C07C
:1021200000E0002391F70FE10E94BC02F1CFE4E050
:102130000C9469329A938A9300E40E94780280E0BA
:1021400008C090E0FC01E45DFC4F04910E94BC02D9
:1021500083958034B0F38991999108950E94583203
:10216000D80180E090E02AC00DE210E0AC010E94AE
:10217000212FF801EA0FFB1FE83601E0F00714F009
:10218000E856F1408F01212F220F220B322F0E949F
:102190001C3045E35AEF6EE87CE30E94DC300E947D
:1021A000CF2EAC01440F551F440F551FFA01E154C7
:1021B000F64D00831183228333830196883000E03B
:1021C000900794F2E4E00C9469320E945832D801EE
:1021D00080E090E02AC00DE210E0AC010E94212FC7
:1021E000F801EA0FFB1FE83601E0F00714F0E856AB
:1021F000F1408F01212F220F220B322F0E941C3021
:1022000045E35AEF6EE87CE30E94DC300E94F23531
:10221000AC01440F551F440F551FFA01E158F64D0C
:1022200000831183228333830196883000E0900776
:1022300094F2E4E00C9469320E945832D80180E0B4
:1022400090E02AC00DE210E0AC010E94212FF801BD
:10225000EA0FFB1FE83601E0F00714F0E856F14002
:102260008F01212F220F220B322F0E941C3045E3B9
:102270005AEF6EE87CE30E94DC300E94CF2EAC0166
:10228000440F551F440F551FFA01E156F64D0083C8
:102290001183228333830196883000E0900794F203
:1022A000E4E00C9469320E945432D80180E090E05E
:1022B00034C08D01212F220F220B322F0E941C309F
:1022C000280139018C01212F220F220B322F0E946D
:1022D0001C304BED5FE069E47FE30E94DC300E943C
:1022E000F235A201B3010E94DC30280139018D01D1
:1022F000212F220F220B322F0E941C30A201B3018A
:102300000E947B300E9429309C01220F331FF9016B
:10231000E159F64D008311830196883000E0900763
:1023200044F2E8E00C9465320E9452324801D9012F
:1023300080E090E046C00DE210E0AC010E94212F49
:10234000A801480D591D483601E0500714F04856C1
:1023500051408D01212F220F220B322F0E941C3061
:10236000280139018A01212F220F220B322F0E94CE
:102370001C300801190145E35AEF6EE87CE3800147
:1023800091010E94DC300E94F235A201B3010E944B
:10239000DC30280139018D01212F220F220B322F31
:1023A0000E941C30A201B3010E947B300E942930A0
:1023B0009C01220F331FF901E15AF64D008311836E
:1023C0000196883000E090070CF4B5CFEAE00C9459
:1023D00063320E94583220E030E000E010E0A4DFD9
:1023E00072D105E00E948903E091B42AF091B52AE8
:1023F000F3970CF4F5C080E09CE5A1ECB7E400E0B5
:1024000010E00093F52A1093F62A08C0E5EFFAE2EF
:10241000008111810B5F1F4F008311830091F52A0A
:102420001091F62A083621E01207BCF520914525C7
:10243000309146250091F52A1091F62A75DF02E0C9
:102440000E9489030091B42A1091B52A212F220FEE
:10245000220B322F0E941C30AC01BD010E94DE31E4
:10246000A8F60091B42A1091B52A212F220F220B31
:10247000322F0E941C30C801D9010091F52A109119
:10248000F62A0093F12A1093F22AE091B42AF091EF
:10249000B52AB8970CF0BACF54C080E09CE5A1EC07
:1024A000B7E405E010E0EED000E010E00093452531
:1024B0001093462508C0E5E4F5E200811181025E33
:1024C0001F4F008311830091452510914625083E3A
:1024D00027E01207B4F5209145253091462500915B
:1024E000F12A1091F22A20DF02E00E948903009174
:1024F000B42A1091B52A212F220F220B322F0E94CD
:102500001C30AC01BD010E94DE31A8F60091B42A56
:102510001091B52A212F220F220B322F0E941C303E
:10252000C801D90100914525109146250093F32A51
:102530001093F42AE091B42AF091B52A74970CF024
:10254000BACFE091F12AF091F22A349744F0E1EF0A
:10255000FAE2008111810350104000831183E09161
:10256000F32AF091F42A369744F0E3EFFAE200817F
:10257000118105501040008311832091F32A30917E
:10258000F42A0091F12A1091F22ACEDE0091F32A6A
:102590001091F42A0093BC2A1093BD2A0091F12ACD
:1025A0001091F22A0093BA2A1093BB2A3091BB2AC9
:1025B000232F0EE010E00E94C80A2091BA2A0FE0F3
:1025C00010E00E94C80A3091BD2A232F00E110E0DC
:1025D0000E94C80A2091BC2A01E110E00E94C80AAA
:1025E0000FEF0093C12AE4E00C94693234E0309399
:1025F00040093091DA2A329F00926A0910926B09E1
:10260000009366091093670908950E945832D80113
:10261000922F24E08D01EADF00E315E756DD88E024
:102620000CC0989F800143E00E94352F202F8D0120
:10263000DDDF00E41CE949DD8A95813090F7E4E0B4
:102640000C9469320E945832D80122E08D01CEDF0D
:1026500008EE1DEF3ADD08EE1DEF37DD84E090E077
:102660000AC0282F8D01C2DF08EE1DEF2EDD08EE17
:102670001DEF2BDD0197813000E0900794F7E4E037
:102680000C94693222E044E650E00E94212FAEDF34
:1026900048E750E00091232A1091242A0E94532FEA
:1026A0000E5F0E94890300E00093400908958A9319
:1026B000812F10E0E7DF00E315E707DD082F10E0CA
:1026C000E1DF899108952CE531E20FE915E20E94DE
:1026D000A53600E80E94180300E310E0D3DF089558
:1026E0000E94672E40E050E064E672E40E94DC3015
:1026F0000E94293008950E94672E40E050E064E671
:1027000072E40E94DC300E9429300B3520E0120771
:1027100014F00BE510E0063A2FEF120714F405EA67
:102720001FEF08950E945432D8012DE631E20FE9DF
:1027300015E20E94A53600E80E941803A13000E0CF
:10274000B00714F180E0082F10E020E030E00E9494
:102750002730280139018D01212F220F220B322F22
:102760000E941C300E947232A801B90182019301BB
:102770000E94DE3178F5082F07570E9478020EE399
:102780000E94BC028395DFCF80E008C006E8081BEA
:102790000E9478020CE30E94BC028395082F10E08F
:1027A00020E030E00E942730280139010FEF1FEFB1
:1027B000AD010E94212F212F220F220B322F0E94C8
:1027C0001C300E947232A801B901820193010E945B
:1027D000DE31E0F200E315E778DCE8E00C946532E6
:1027E0000E945832A0E0B0E000E00093010204E053
:1027F0000E94890380E090E019C0E0E0F2E00081EF
:102800000860008300912B020023E1F301E00093B4
:102810002B020091120210911302A00FB11F009120
:10282000E82A1091E92AA01BB10B0196803A00E03A
:1028300090071CF300E10093010200E117E245DC80
:10284000BB2312F4A0E0B0E040E650E08D010E940E
:10285000532FE4E00C9469320E94583280E090E0FB
:1028600000E00093010203E00E948903A0E0B0E0D1
:1028700013C0E0E0F2E000810860008300912B02C9
:102880000023E1F301E000932B020091120210916A
:102890001302800F911F1196A43600E0B0074CF38D
:1028A00000E10093010244E650E08C010E94532FA6
:1028B000E4E00C946932E0E0F2E000810061008322
:1028C000009133020023E1F301E0009333024091D1
:1028D000D52A50E000911402109115020E943B2F5E
:1028E00008950091B62A1091B72A6FDC0091B62A9C
:1028F0001091B72AA1DC0091B62A1091B72A009353
:10290000B82A1093B92A0091B82A1091B92A26DC66
:1029100008950091B62A1091B72A57DC0091B62A83
:102920001091B72A89DC0091B82A1091B92A16DCD7
:102930004091E02A50E00FEF10E00E94212FB3DC1D
:102940000091232A1091242A009326091093270925
:1029500008959A938A9301E010E00E947E0A902FD6
:1029600080E002E010E00E947E0A10E0802B912BB4
:102970008093232A9093242A05E010E00E947E0A87
:10298000902F80E006E010E00E947E0A10E0802B8D
:10299000912B8093B62A9093B72A07E010E00E940B
:1029A0007E0A902F80E008E010E00E947E0A10E08E
:1029B000802B912B8093B82A9093B92A0EE010E0D7
:1029C0000E947E0A902F80E00FE010E00E947E0AB5
:1029D00010E0802B912B8093BA2A9093BB2A00E1C0
:1029E00010E00E947E0A902F80E001E110E00E943A
:1029F0007E0A10E0802B912B8093BC2A9093BD2AF5
:102A000003E010E00E947E0A0093D12A04E010E067
:102A10000E947E0A0093D22A09EF11E00E947E0AEA
:102A20000093D42A07EF11E00E947E0A0093DD2A6A
:102A30000CE010E00E947E0A0093E02A0DE010E016
:102A40000E947E0A0093DC2A0BEF11E00E947E0AAE
:102A50000093E32A0CEF11E00E947E0A0093D52A2E
:102A600006EF11E00E947E0A0093DA2A05EF11E0DA
:102A70000E947E0A0093E12A0DEF11E00E947E0A77
:102A80000093DB2A02E110E00E947E0A0093DF2A15
:102A90000AE010E00E947E0A802F90E00BE010E038
:102AA0000E947E0A102F00E0802B912B8093E42A55
:102AB0009093E52A03E110E00E947E0A0093E22A47
:102AC00008EF11E00E947E0A0093C72A0EEF11E082
:102AD0000E947E0A0093CF2A04E110E00E947E0A41
:102AE0000093D02AE4EEFAE200810160008389912C
:102AF000999108950E945832D801AB3500E0B00793
:102B000014F0AAE5B0E00091CC2A002331F0009146
:102B1000E22A033011F088E40DC0BB2312F48CE3E9
:102B200009C04AE050E08D010E94532F102F06E0AB
:102B3000109F802D00E80E94780290E0FC01E4598B
:102B4000FC4F04910E94BC0201E80E94780290E0D0
:102B5000FC01E359FC4F04910E94BC0202E80E9470
:102B6000780290E0FC01E259FC4F04910E94BC0203
:102B700000EC0E94780290E0FC01E159FC4F0491C6
:102B80000E94BC0201EC0E94780290E0FC01E05936
:102B9000FC4F04910E94BC0202EC0E94780290E07B
:102BA000FC01EF58FC4F04910E94BC020091CC2A1A
:102BB000002331F00091E22A033011F088E40CC0C8
:102BC000BB2312F482E408C04AE050E08D010E9469
:102BD000532F06E0409F802D04E80E94780290E089
:102BE000FC01E459FC4F04910E94BC0205E80E94DC
:102BF000780290E0FC01E359FC4F04910E94BC0272
:102C000006E80E94780290E0FC01E259FC4F049132
:102C10000E94BC0204EC0E94780290E0FC01E159A1
:102C2000FC4F04910E94BC0205EC0E94780290E0E7
:102C3000FC01E059FC4F04910E94BC0206EC0E948A
:102C4000780290E0FC01EF58FC4F04910E94BC0216
:102C500003E80E94780200E20E94BC0203EC0E949A
:102C6000780200E20E94BC02E4E00C9469320E9407
:102C70005832E4EEFAE2018107FF02C005E501C027
:102C800008E530912C2A33230AF47DC020912B2AA9
:102C900030912C2A10E0201731070CF074C04AE064
:102CA00050E00091252A1091262A0E94532F402F90
:102CB0004A5F0091E42A1091E52A0E94352F0170A5
:102CC000002309F060C00091DD2A013031F4209129
:102CD000C62A00E717E18ADCB0C00091DD2A023085
:102CE00001F5E091252AF091262A759734F4209178
:102CF000C62A00EE1EE27ADCA0C00091252A1091BF
:102D0000262A0B3420E0120734F02091C62A00EA6C
:102D10001FE06CDC92C02091C62A00E717E166DC58
:102D20008CC00091DD2A0330B9F42091C62AA22F6D
:102D30008AE090E04AE050E00091252A1091262A8E
:102D40000E94532F801B910B00E416E0AC010E94FF
:102D5000212F2A2F4BDC71C02091C62AA22F8AE096
:102D600090E04AE050E00091252A1091262A0E9426
:102D7000532F801B910B00E416E0AC010E94212F21
:102D80002A2F43DC5AC01091262A11230AF055C07D
:102D90000091D22A10E020E030E00E942730C801E4
:102DA000D90103E010E04091212A5091222A0E948B
:102DB000212F212F220F220B322F0E941C300E9424
:102DC0007232A801B9018C019D010E94DE31A8F583
:102DD00084E04CEE5FEF0091252A1091262A0E9494
:102DE000532F801B482F0091E42A1091E52A0E945E
:102DF000352F0170002309F50091252A1091262A0C
:102E00000093292A10932A2A43E00091C62A0E949F
:102E1000032F0093C62A0091252A1091262A063FE7
:102E20002FEF12072CF02091C62A00E516E4DEDB16
:102E30002091C62A00E61DE6D9DBE4E00C94693255
:102E40009A938A938091232A9091242A0196AC0127
:102E5000652F660F660B762F00E01CE62CED32E046
:102E60000E94BA2F43E00E948F2F48E050E060E0BC
:102E700070E00E94672F40E750E060E070E00E9441
:102E8000BA2F0093332A1093342A45E00091332A55
:102E90001091342A0E942F2F40E250E00E94212FEF
:102EA0000093332A1093342A0091332A1091342A44
:102EB000000F012F001F10E0111F0093352A1093FF
:102EC000362A0091E22A0130A9F40091332A1091A8
:102ED000342A0093312A1093322A4AE150E00091BB
:102EE000232A1091242A0E94532F0093372A1093EB
:102EF000382A16C00091332A1091342A000F111F6E
:102F00000093312A1093322A40E150E00091232AA5
:102F10001091242A0E94532F0093372A1093382AA5
:102F20000091CC2A002321F40091E22A033041F4DD
:102F30000091CC2A002359F00091E22A033039F4A1
:102F400001E010E00093392A10933A2A06C000E00D
:102F500010E00093392A10933A2A899199910895A3
:102F60008A930091CF2A10E0F801E654FC4F0491B7
:102F7000002351F10091CA2A002331F59CDC2091F5
:102F8000CF2A30E0F901E654FC4F249130E00217DB
:102F90001307D4F480E016C02EE731E20FE915E202
:102FA0000E94A53600E80E94180308E710E06ADBDB
:102FB00008EE1DEF8AD801E00E94780202E00E942C
:102FC00089038395853040F3899108951091E22A11
:102FD000133009F4039510912002137E1093200200
:102FE0000A95000F000F10912002102B1093200261
:102FF0000895AFDC25DF0E9446020091E12A0230ED
:1030000031F40091CA2A002311F494D801C06ED87B
:103010002091BC2A3091BD2A0091BA2A1091BB2A76
:1030200083D977DC0091DF2AD1DF08959A938A93C0
:10303000F89410E500E33BDBDCDF01E00E9478025E
:1030400000E117E20E9465108091232A9091242AC2
:103050000196AC01652F660F660B762F00E01CE62B
:103060002CED32E00E94BA2F43E00E948F2F1A937A
:103070000A932FE831E20FE915E20E94A536229665
:1030800000E80E941803789400E00093CC2A00E046
:1030900010E00093292A10932A2A0093272A1093DC
:1030A000282A01E010E00093E62A1093E72A01E0C5
:1030B0000093C22A04EB0093CE2A0093CD2A00E0AD
:1030C00010E020E030E0EFE7FAE200831183228392
:1030D0003383E3E7FAE20083118322833383E7E556
:1030E000FAE200831183228333830091372A102F61
:1030F00003E0109F002D0E94890389919991089502
:103100000E944C322197F894A0E005C00A2F10E0ED
:103110000E94E510A395AC30C8F300E30E941D03A4
:10312000E0E8F6E0008108600083009160060F602F
:103130000093600600914006006C00934006E0E6B4
:10314000F6E0008100620083E0E4F6E000810260C6
:10315000008300916006006C0093600608E1009314
:10316000110608E10093120608E10093130608E136
:103170000093300608E10093520608E100935306DD
:103180000E9446020AEF11E00E947E0A0F3F11F4EE
:1031900001E001C000E0E8E0F6E0108111FD0CC0A4
:1031A000E8E0F6E0108112FD07C0E8E2F6E02081D9
:1031B000217011E0212701C020E0022B002309F437
:1031C000CAC020EA31E20FE915E20E94A53600EC00
:1031D0000E941803789402E30E948903F89400E0A7
:1031E0000093EF2A05C00091EF2A03950093EF2A80
:1031F0000091EF2A033008F0A9C000E00093EE2A06
:1032000013C0B0E0FD01E352FC4F24910A2F10E0FF
:1032100000541E4F0E94C80AA395A93090F3009154
:10322000EE2A03950093EE2A0091EE2A0330D8F699
:1032300022E001E010E00E94C80A27E502E010E069
:103240000E94C80A20E005E010E00E94C80A24EBB2
:1032500006E010E00E94C80A20E007E010E00E94AB
:10326000C80A20ED08E010E00E94C80A20E00EE045
:1032700010E00E94C80A20E00FE010E00E94C80A97
:1032800020E000E110E00E94C80A20E001E110E027
:103290000E94C80A22E003E010E00E94C80A22E06F
:1032A00004E010E00E94C80A20E009EF11E00E944B
:1032B000C80A27E00CE010E00E94C80A21E00DE0F7
:1032C00010E00E94C80A21E007EF11E00E94C80A3E
:1032D00021E00AE010E00E94C80A20E80BE010E0BC
:1032E0000E94C80A20E00BEF11E00E94C80A28E102
:1032F0000CEF11E00E94C80A27E006EF11E00E94DF
:10330000C80A26E00DEF11E00E94C80A22E002E19F
:1033100010E00E94C80A21E005EF11E00E94C80AEF
:1033200021E003E110E00E94C80A20E008EF11E06C
:103330000E94C80A22E00EEF11E00E94C80A24E0B1
:1033400004E110E00E94C80AA0E067CF20E00AEF85
:1033500011E00E94C80A00E00093EF2A009148069D
:103360000C700093F02A0091F02A0C3021F401E057
:103370000093EE2A0FC00091F02A083021F400E0FB
:103380000093EE2A07C00091F02A043019F402E0FD
:103390000093EE2A2EDE02E00093D22A02E0009390
:1033A000D12A01E00093DC2A0091C72A023019F4E7
:1033B00000E00093C72A03E20093010807E00093AE
:1033C000000806E910E00093260810932708809172
:1033D000DB2A90E0019680932A0890932B080091B5
:1033E000DB2A002331F400E010E00093260810935C
:1033F000270801E0009300090091232A1091242A54
:10340000009326091093270903E000930609009111
:10341000A20007600093A20007E00093400804EDBB
:1034200011E0009366081093670801E000934608D6
:103430000E946F032091BC2A3091BD2A0091BA2AC4
:103440001091BB2A0E9494110E94460302E000934F
:1034500022020E9468030E9461030E9446030091B9
:10346000DF2AB4DD56DA02E00E948903F5D9009321
:10347000E82A1093E92A03E20093410900916406C7
:103480000F730093640622EB31E20FE915E20E940C
:10349000A53600EC0E94180300E210E01A930A938C
:1034A00023EC31E20FE915E20E94A536229600E8EE
:1034B0000E94180300ED17E0C5D800EA1FE0C2D84B
:1034C00000E41FE1BFD808EE1DEF0E94651000ED7B
:1034D00017E0B8D800E00093400900E000934009ED
:1034E0000091372A102F05E0109F002D0E948903BC
:1034F00000919F250B3409F0BECF0091A025003527
:1035000009F0B9CF0091A1250F3409F0B4CF009193
:10351000D42A002331F0009164060F7300936406EF
:1035200005C000916406006C009364060091A2251A
:10353000043509F0A0CF78940CE00E94780202E0F4
:103540000E9489030DDDE8E0F6E0008101FD23C063
:10355000E8E0F6E0008102FD1EC00FEF0093CA2AEA
:1035600001E00093C92A01E00093CB2A01E00E9408
:10357000780210E500E39BD825ED31E20FE915E272
:103580000E94A53600E80E941803E8E0F6E00081FA
:1035900002FFFBCF52C1E8E0F6E0008102FD21C04E
:1035A0000FEF0093CA2A0BE00093C92A02E00093B0
:1035B000CB2A01E00E94780210E500E30E94571335
:1035C00026EE31E20FE915E20E94A53600E80E94DE
:1035D0001803E8E0F6E0008102FFFBCF0E947610BE
:1035E0002CC100E00093CB2A00E61AEE0E94651081
:1035F000F7D838010091372A102F02E0109FA02D34
:1036000055C04091232A5091242A4F5F5F4F652F68
:10361000660F660B762F00E01CE62CED32E00E9470
:10362000BA2F43E00E948F2FC8017A926A929A9330
:103630008A9320E232E20FE915E20E94A536249631
:1036400000E80E9418030091B42A1091B52A1A9339
:103650000A932FE232E20FE915E20E94A536229684
:1036600000EC0E9418030091E22A10E0000F111FE5
:10367000F801EB53FC4F059114911A930A930091B2
:10368000DF2A10E0F801E154FC4F049110E01A9396
:103690000A932BE332E20FE915E20E94A536249645
:1036A00009EC0E94180302E00E9489030A2FA02F50
:1036B000AA95002309F050C001E00E94780200E2C0
:1036C0001EE40E94651005E0601600E070060CF034
:1036D00083C024E432E20FE915E20E94A53600E837
:1036E0000E94180300ED10E00E94421300EB10E06E
:1036F0000E94421300ED10E00E94421304E10E9478
:1037000089039BC081E090E00091DF2A10E0F8017E
:10371000E154FC4F049110E01A930A930091B62AE9
:103720001091B72A2091B82A3091B92A021B130BA5
:103730001A930A939A938A93B0E0BA93AA932AE0D1
:1037400032E20FE915E20E94A536289600EC0E94AD
:10375000180308E00E948903E8E2F6E0008100FD1A
:1037600050CF0AE00E9489038090B42A9090B52A35
:103770000091DE2A10E01A930A937A926A929A9242
:103780008A9227EF31E20FE915E20E94A5362696CC
:1037900000E80E9418030091E42A1091E52A013004
:1037A00020E8120761F000E02091E42A3091E52A38
:1037B000213010E0310719F00060002311F0A0E083
:1037C00001C0A1E00091BC2A1091BD2A012B09F093
:1037D00099CF80E090E098CF0091B42A1091B52A5B
:1037E000093522E012074CF125E532E20FE915E236
:1037F0000E94A53600EC0E94180300ED10E00E9424
:10380000421300EB10E00E94421300ED10E00E9412
:103810004213A1E010C008EE1DEF0E946510E8E021
:10382000F6E0008102FD06C00E94E91110E200E30B
:103830000E945713A395A93170F301E00093C22AA7
:1038400000E00093D62A07E00093CE2A0093CD2A09
:1038500000E010E020E030E0EFE7FAE200831183BF
:1038600022833383E3E7FAE20083118322833383E5
:103870000093292A10932A2A0093272A1093282A92
:10388000212F220F220B322FE7E5FAE2008311836A
:103890002283338301E010E00093E62A1093E72AA5
:1038A00005E00E94890300E310E00E94421302E059
:1038B0000E94890300E310E00E9442130E94F0136B
:1038C0004091B42A5091B52A0E94212FC8018F7FC0
:1038D0009070863600E0900731F52FEF0AEF11E087
:1038E0000E94C80A20C00091F02A043019F402E0B6
:1038F0000093EE2A9BDB01E0C00E00E0D01E8601A3
:10390000680101342FE1120774F0CC24DD2428DB98
:103910000091BE2A1091BF2A083522E012071CF43C
:1039200001E00093C22A0091CA2A002309F07BC358
:103930000091392A10913A2A013020E0120709F04B
:103940005FC1E7E4FAE20081118122813381EBE675
:10395000FAE20083118322833383EBE4FAE20081ED
:10396000118122813381E7E7FAE200831183228308
:103970003383E7E5FAE2008111810093212A109355
:10398000222A0091D12A0093D32A0091DC2A013007
:1039900029F40091D32A0E5F0093D32A0091D32AF1
:1039A00010E02091212A3091222A021713070CF0EF
:1039B000EAC00091C92A002309F0E5C000E00093A5
:1039C000CD2A0091CE2A03950093CE2AEFE6FAE2A3
:1039D0000081118122813381EBE6FAE2408151813D
:1039E00062817381401B510B620B730B40835183C7
:1039F00062837383EBE7FAE20081118122813381D4
:103A0000E7E7FAE24081518162817381401B510BEB
:103A1000620B730B4083518362837383EBE6FAE29C
:103A20000081118122813381EBE6FAE240815181EC
:103A3000628173810E94672FC801D901E7E7FAE22A
:103A40000081118122813381E7E7FAE240815181CF
:103A5000628173810E94672FA801B9018C019D01C9
:103A6000040F151F261F371F0E941C300E94C036EE
:103A70000E94293028015594479455944794552025
:103A80004AF422E104EF1EE70E94F61200E21EE46F
:103A90000E946510E7E7FAE20081118122813381FB
:103AA0000E941C30A801B901CA01DB01EBE6FAE271
:103AB00000811181228133810E941C30AC01BD0143
:103AC0000E947B130093252A1093262A0091212A15
:103AD0001091222A212F220F220B322F0E941C30FC
:103AE0000E9472320E94293003950093C62A0091E9
:103AF000C72A013021F408E00093C62A0AC00091C9
:103B0000C72A023031F40AE01091C62A011B009343
:103B1000C62A0091DD2A043089F00091C62A10914E
:103B2000C62A019F800149E050E02091DA2A30E066
:103B3000421B530B0E94532F0093C62A0091212A47
:103B40001091222AE016F10684F40091252A1091A2
:103B5000262A00932B2A10932C2A4092E62A509270
:103B6000E72AE090212AF090222A00912B2A109136
:103B70002C2A0093292A10932A2A0093252A10938D
:103B8000262A75D850C200E010E000936A0910930D
:103B90006B09EBE6FAE20081118122813381EFE6C5
:103BA000FAE20083118322833383E7E7FAE200819C
:103BB000118122813381EBE7FAE2008311832283B2
:103BC0003383EE24FF240091CD2A03950093CD2A60
:103BD00000E00093CE2A4AE00091CD2A0E94032FF4
:103BE000442309F020C20091BE2A1091BF2A0D3D46
:103BF00025E012070CF417C201E00093C22A13C299
:103C00000091CC2A002309F023C10091E22A03305D
:103C100009F01EC1E7E4FAE20081118122813381BB
:103C2000E3E7FAE24081518162817381041B150B45
:103C3000260B370BEBE6FAE20083118322833383F2
:103C4000EBE4FAE20081118122813381EFE7FAE2AD
:103C50004081518162817381041B150B260B370B48
:103C6000E7E7FAE20083118322833383E7E5FAE290
:103C7000008111810093212A1093222AEBE4FAE2B9
:103C800000811181228133810E941C30A801B90179
:103C9000CA01DB01E7E4FAE200811181228133816C
:103CA0000E941C30AC01BD010E947B130093252AA9
:103CB0001093262A0091252A1091262A053A2FEFE3
:103CC000120761F000E02091252A3091262A2B3539
:103CD00010E0310719F00060002341F00091292A1B
:103CE00010912A2A0093252A1093262AEBE6FAE25D
:103CF0000081118122813381EBE6FAE2408151811A
:103D0000628173810E94672FC801D901E7E7FAE257
:103D10000081118122813381E7E7FAE240815181FC
:103D2000628173810E94672FA801B9018C019D01F6
:103D3000040F151F261F371F0E941C300E94C0361B
:103D40000E94293045E00E94352F280155204AF471
:103D500022E100E01DE70E94F61200E41CE90E9447
:103D60006510088103950883053128F001E0009370
:103D7000C22A00E008830091212A1091222A0F5FB5
:103D80001F4F212F220F220B322F0E941C300E9426
:103D900072320E9429300093C62A0091C62A1091DF
:103DA000C62A019F0092C62A0091C62A10E049E067
:103DB00050E02091DA2A30E0421B530B0E94532F2F
:103DC00003950093C62A042D052939F442E0009199
:103DD000C62A0E94032F0093C62A04E000934009DC
:103DE0000091DA2A06951091C62A019F00926A096D
:103DF00010926B09E091212AF091222A32978CF0DF
:103E00001091262A11236AF000E41FE12091212A53
:103E10003091222A021B130B009366091093670945
:103E20000AC00091212A1091222A005C104E0093B2
:103E30006609109367094092E62A5092E72A00919A
:103E4000252A1091262A0093292A10932A2AEBC0AA
:103E50004091DF2A50E060E070E0E7E4FAE20081A0
:103E60001181228133810E94BA2FEBE6FAE20083AE
:103E70001183228333834091DF2A50E060E070E0B9
:103E8000EBE4FAE200811181228133810E94BA2F92
:103E9000E7E7FAE200831183228333834091DF2A2C
:103EA00050E060E070E0E7E5FAE2008111812281F4
:103EB00033810E94BA2F0093212A1093222AEBE625
:103EC000FAE20081118122813381EBE6FAE240813E
:103ED0005181628173810E94672FC801D901E7E790
:103EE000FAE20081118122813381E7E7FAE2408121
:103EF0005181628173810E94672FA801B9018C01F1
:103F00009D01040F151F261F371F0E941C300E94A1
:103F1000C0360E94293028015594479455944794FF
:103F20008091D12A90E001960091212A1091222AB5
:103F3000801791070CF06CC00091C92A002309F08A
:103F400067C00091CE2A03950093CE2A00E000932B
:103F5000CD2A55204AF422E100E01DE70E94F61226
:103F600000E41CE90E9465100091212A1091222A88
:103F70000F5F1F4F212F220F220B322F0E941C3068
:103F80000E9472320E9429300093C62A0091C62AEC
:103F90001091C62A019F800149E050E02091DA2A61
:103FA00030E0421B530B0E94532F0093C62A00910E
:103FB000CE2A043060F02091C62A00E41FE140912F
:103FC000212A5091222A041B150B0E94F6124092BE
:103FD000E62A5092E72AE7E7FAE20081118122817E
:103FE00033810E941C30A801B901CA01DB01EBE654
:103FF000FAE200811181228133810E941C30AC01E0
:10400000BD010E947B130093292A10932A2A0BC01A
:1040100000E00093400900E00093CE2A0091CD2AF1
:1040200003950093CD2A0091CD2A0C3D41F010E07C
:104030000091CE2A0C3D19F01060112389F000E0A8
:1040400010E00093E62A1093E72A0093292A1093A0
:104050002A2A0093272A1093282A01E00093C22AD3
:104060000091C92AE6EEF3E00C9407328091292AE8
:1040700090912A2AE091E62AF091E72A33972CF0D2
:104080008093272A9093282A04C08091272A909110
:10409000282A0091E12A023009F080C08C010E9498
:1040A0007A1504E610E00E9465100091E62A10914E
:1040B000E72A212F220F220B322F0E941C300E9450
:1040C00072320E942930C8010091CD2A053048F093
:1040D00026E632E20FE915E20E94A53607EC0E94BF
:1040E0001803552032F403E2802E992489E090E0F1
:1040F0000DC00091392A10913A2A012B21F40EE3C8
:10410000802E992403C006E0802E9924A0E008C0E8
:104110000A2F08530E947802082D0E94BC02A39522
:10412000B0E0A817B907A4F30091B32A10E01A93DE
:104130000A930091DC2A10E01A930A930091D12A85
:1041400010E01A930A930091D22A10E01A930A936E
:1041500020E732E20FE915E20E94A536289607E82B
:104160000E9418030E945B1448014AE050E0840159
:104170000E94532F5A934A934AE050E084010E94D0
:10418000532F1A930A932BE732E20FE915E20E94AC
:10419000A53624960DE80E941803E1C4992352F035
:1041A0009A938A9322E832E20FE915E20E94A5363B
:1041B00022960EC04FEF5FEF8C010E94212F1A93C1
:1041C0000A9329E832E20FE915E20E94A536229609
:1041D00000E80E9418030091E62A1091E72A212F97
:1041E000220F220B322F0E941C300E9472320E943A
:1041F0002930C80199231AF483E290E006C0883080
:1042000000E0900711F48FEF90E004E80E9478023C
:10421000082F0E94BC020091B32A10E01A930A935F
:104220000091DC2A10E01A930A930091D12A10E041
:104230001A930A930091D22A10E01A930A9320E964
:1042400032E20FE915E20E94A536289605E80E94A1
:1042500018030E945B1448014AE050E084010E9468
:10426000532F5A934A934AE050E084010E94532FFF
:104270001A930A932DE932E20FE915E20E94A5365E
:1042800024960DE80E9418030091392A10913A2AC9
:10429000013020E0120709F04FC00091CD2A06300E
:1042A00048F023EA32E20FE915E20E94A53600EC5D
:1042B0000E941803E091252AF091262A31977CF07C
:1042C0000091252A1091262A045C1F4F4AE050E0F5
:1042D0000E94532F00932D2A10932E2A12C042E0E1
:1042E00050E00091252A1091262A0E94532F0E5C3F
:1042F0001F4F4AE050E00E94532F00932D2A109345
:104300002E2A00912D2A00540E947802813000E06C
:1043100090075CF00091CD2A013020F006E00E9469
:10432000BC0203C004E00E94BC0205EC0E947802BB
:104330000FE20E94BC0213C443E082010E94352FA9
:10434000C801833C01E0900734F400E099231AF09F
:104350000060002311F082EC91E024EB32E20FE9DF
:1043600015E20E94A53600EC0E941803A0E00FC0E1
:104370000A2F07530E9478020EE30E94BC0206EC4B
:104380000A1B0E9478020CE30E94BC02A3950A2F2C
:1043900010E020E030E00E942730480159018C01F4
:1043A000212F220F220B322F0E941C300E947232CA
:1043B000A801B901840195010E94DE31C8F200ED27
:1043C00017E00E946510CBC38091EE2A90E0019621
:1043D0009A938A9325EC32E20FE915E20E94A53602
:1043E000229600E80E94180307E80E947802A0E0E5
:1043F00009C00A2F10E000541E4F0E947E0A0E943E
:10440000BC02A395A930A8F300E21EE40E94651047
:10441000E8E2F6E0008100FD0BC008E210E00E9437
:1044200042130DE00E947802A0E407E00093D62A30
:104430000E9476102EEC32E20FE915E20E94A536BA
:1044400000EC0E941803A0E010C00A2F0A530E943B
:1044500078020A2F0E94BC02A83031F40EEC0E94B0
:1044600078020FEF0E94BC02A3958091EE2A90E0A3
:104470000196B0E08A179B0744F771C30E945B1452
:10448000C8014AE050E08C010E94532F5A934A938E
:104490004AE050E08C010E94532F1A930A93009136
:1044A000CF2A10E0F801E654FC4F04914AE00E9444
:1044B000032F50E05A934A930091CF2A10E0F8015D
:1044C000E654FC4F04914AE00E94032F10E01A9337
:1044D0000A9320EE32E20FE915E20E94A5362896F3
:1044E00000E80E9418030091D52A10E01A930A935D
:1044F00026EF32E20FE915E20E94A536229600EC83
:104500000E94180302E00E94890329C30091DB2A5C
:1045100010E01A930A9327E033E20FE915E20E94B4
:10452000A536229600E80E94180329E133E20FE93C
:1045300015E20E94A53600EC0E941803A0E010C00E
:104540000A2F0A530E9478020A2F0E94BC02A83048
:1045500031F40EEC0E9478020FEF0E94BC02A3958A
:104560000091DB2A0A1760F702E00E948903F7C274
:104570000E94F013C8019A938A932BE233E20FE969
:1045800015E20E94A536229600E80E9418030091C9
:10459000312A1091322A1A930A932EE333E20FE95B
:1045A00015E20E94A536229609E80E941803409160
:1045B000232A5091242A4F5F5F4F652F660F660BA9
:1045C000762F00E01CE62CED32E00E94BA2F43E08B
:1045D0000E948F2F3A932A931A930A9327E433E287
:1045E0000FE915E20E94A536249600EC0E941803FC
:1045F00000E21EE40E946510B2C240E250E060E0BA
:1046000070E0EBE4FAE200811181228133810E94A3
:10461000BA2F0E94921327E533E20FE915E20E94B8
:10462000A53600EC0E9418030FED10E01A930A93D0
:104630000091B62A1091B72A1A930A9322E633E220
:104640000FE915E20E94A53624960AEC0E94180391
:1046500000E21EE40E94651082C244E050E060E087
:1046600070E0E7E5FAE200811181228133810E9446
:10467000BA2F0E9492132BE633E20FE915E20E9453
:10468000A53600EC0E9418030FED10E01A930A9370
:104690000091B82A1091B92A1A930A9322E633E2BC
:1046A0000FE915E20E94A53624960AEC0E94180331
:1046B00000E41CE90E94651052C20091C72A10E074
:1046C000000F111FF801E153FC4F059114911A934B
:1046D0000A9327E733E20FE915E20E94A5362296F6
:1046E00000E80E9418032EE733E20FE915E20E946A
:1046F000A53606E80E94180329E833E20FE915E21F
:104700000E94A53600EC0E941803A0E010C00A2FFA
:104710000A530E9478020A2F0E94BC02A83031F48A
:104720000EEC0E9478020FEF0E94BC02A39500914C
:10473000DA2A0A1760F700E61AEE0E9465100FC227
:104740000091DD2A033019F48AE090E005C08091E1
:10475000DD2A90E0880F991F0091DD2A043039F49A
:104760002AE933E20FE915E20E94A53609C09A93BF
:104770008A9321EA33E20FE915E20E94A5362296D8
:1047800000E80E9418032EE733E20FE915E20E94C9
:10479000A53606E80E94180329EA33E20FE915E27C
:1047A0000E94A53600EC0E941803A0E010C00A2F5A
:1047B0000A530E9478020A2F0E94BC02A83031F4EA
:1047C0000EEC0E9478020FEF0E94BC02A3950091AC
:1047D000DD2A0A1760F702E00E9489030091DD2AB2
:1047E000053081F48EE591E009C08093260990930D
:1047F000270908EB1BE00E9465100496883E03E041
:1048000090079CF3ACC10091E12A10E0000F111F4A
:10481000F801ED52FC4F059114911A930A932AEB7B
:1048200033E20FE915E20E94A536229600E80E94C5
:10483000180329EC33E20FE915E20E94A53600ECDB
:104840000E941803A0E010C00A2F0A530E947802A9
:104850000A2F0E94BC02A83031F40EEC0E947802AC
:104860000FEF0E94BC02A3950091E12A0A1760F79E
:1048700002E00E94890373C10091E22A10E0000F58
:10488000111FF801EB53FC4F059114911A930A93F1
:104890002BED33E20FE915E20E94A536229600E8DF
:1048A0000E94180329EE33E20FE915E20E94A536B3
:1048B00000EC0E941803A0E010C00A2F0A530E94C7
:1048C00078020A2F0E94BC02A83031F40EEC0E943C
:1048D00078020FEF0E94BC02A3950091E22A0A170A
:1048E00060F702E00E9489033AC10E94F0131A9314
:1048F0000A932BEF33E20FE915E20E94A5362296C8
:1049000000E80E9418032EE733E20FE915E20E9447
:10491000A53606E80E94180323E034E20FE915E209
:104920000E94A53600EC0E941803A0E010C00A2FD8
:104930000A530E9478020A2F0E94BC02A83031F468
:104940000EEC0E9478020FEF0E94BC02A39500912A
:10495000E02A0A1760F702E00E94890300C1009173
:10496000DF2A10E0F801E154FC4F049110E01A93A3
:104970000A9324E134E20FE915E20E94A53622965B
:1049800000E80E9418032EE733E20FE915E20E94C7
:10499000A53606E80E9418032CE134E20FE915E27F
:1049A0000E94A53600EC0E941803A0E010C00A2F58
:1049B0000A530E9478020A2F0E94BC02A83031F4E8
:1049C0000EEC0E9478020FEF0E94BC02A3950091AA
:1049D000DF2A0A1760F702E00E948903C0C0009135
:1049E000B42A1091B52A1A930A932DE234E20FE902
:1049F00015E20E94A536229600E80E941803009155
:104A0000BC2A1091BD2A1A930A9328E334E20FE9D5
:104A100015E20E94A536229609E80E9418030FEDC0
:104A200010E01A930A930091BA2A1091BB2A1A93A4
:104A30000A9321E434E20FE915E20E94A536249698
:104A400000EC0E9418030091C12A002321F409E818
:104A50000E94780203C009EC0E9478020EE30E94D3
:104A6000BC0202E00E9489037AC00091D02A10E0C3
:104A70001A930A9324E534E20FE915E20E94A53661
:104A8000229600E80E9418032EE733E20FE915E2B0
:104A90000E94A53606E80E9418032CE534E20FE9CF
:104AA00015E20E94A53600EC0E941803A0E010C099
:104AB0000A2F0A530E9478020A2F0E94BC02A830D3
:104AC00031F40EEC0E9478020FEF0E94BC02A39515
:104AD0000091D02A0A1760F702E00E94890301E0E2
:104AE0000093C42A3CC00091C42A0023C1F12DE6E2
:104AF00034E20FE915E20E94A53600E80E9418038F
:104B0000A0E004C000E20E94BC02A395A03190F492
:104B10000A2F00540E9478024A2F0091E42A109133
:104B2000E52A0E94352F0170002361F303E20E9401
:104B3000BC02EBCF05EC0E9478020FE20E94BC029F
:104B40000091D62A00540E9478020EE00E9478025A
:104B500000E00093C42A08EE1DEF0E946510B0E04B
:104B6000E8E0F6E0008103FDC7C000E000934009E3
:104B700001E00093C22A0091C82A0130B1F406E294
:104B800010E00E944213E8E0F6E0008103FFFBCF53
:104B900001E00093C22A04EB0093CE2A0093CD2AB1
:104BA00000E00093C82A0C942C2EE8E0F6E0008187
:104BB00003FD54C008EE1DEF0E946510B3950B2F46
:104BC000B02F2091372A3091382A10E02017310772
:104BD00060F70091CA2A00950093CA2A01E0009369
:104BE000C82A0091E12A023019F40E949A1002C0EA
:104BF0000E94761001E00E9478020091CA2A0023E8
:104C000081F400E00093C92A4091E02A50E00FEFC0
:104C100010E00E94212F0E94531102E00E9489039C
:104C20000CC007E00093C92A02E00E94890300E05B
:104C300010E00E9453110E94761001E00093C42AF4
:104C400000E00093CB2A00E00093CC2A0AE510E0B4
:104C50000E94421301E00093C22A8EC10091CA2A29
:104C6000002369F40091CC2A00950093CC2A0E947D
:104C7000201704EB0093CE2A0093CD2A38C00CE015
:104C80000E9478020091CB2A013059F40091C92A80
:104C900003950093C92A0730E8F001E00093C92A80
:104CA00019C00091CB2A023059F40091C92A03950A
:104CB0000093C92A003170F00BE00093C92A0AC0A2
:104CC0000091C92A03950093C92A003118F001E028
:104CD0000093C92A0091C92A083049F44091E02A7A
:104CE00050E00FEF10E00E94212F0E94531108E2C4
:104CF00010E00E944213ADC7E8E2F6E0008100FD3B
:104D000076C300E0009340090091C92A0050B1F039
:104D1000025009F43BC1025009F453C10A9509F449
:104D20009AC10A9509F49BC20A9509F4D4C20650A7
:104D300009F4EAC2025009F413C351C301E00E940E
:104D4000780200E21EE40E946510E8E2F6E00081CD
:104D500000FD0FC000E61AEE0E946510B3950B2F00
:104D6000B02F2091372A3091382A10E020173107D0
:104D700060F7B3950B2FB02F2091372A3091382A46
:104D800010E02017310708F0C8C000E310E00E94CF
:104D90004213E3E5FAE200811181228133810E940E
:104DA0001C30A801B901CA01DB01EFE4FAE200817D
:104DB0001181228133810E941C30AC01BD010E940F
:104DC0007B130093252A1093262AEFE4FAE2008150
:104DD000118122813381E3E7FAE200831183228388
:104DE0003383E3E5FAE20081118122813381EFE729
:104DF000FAE200831183228333838201212F220F61
:104E0000220B322F0E941C300E9472324091252AC0
:104E10005091262A5A934A9340E050E060E070E4B3
:104E20000E94DC300E9429301A930A932EE734E264
:104E30000FE915E20E94A536249600E80E941803A7
:104E40000091252A1091262A0F3C2FEF120764F4B7
:104E500000E02091252A3091262A263A1FEF3107BB
:104E60001CF000600023D9F023E934E20FE915E2D9
:104E70000E94A53600EC0E94180300EA10E00E9490
:104E8000421300EB10E00E944213E8E2F6E00081DA
:104E900000FD63C0E8E0F6E0008103FDF6CF24EA00
:104EA00034E20FE915E20E94A53600EC0E941803D7
:104EB00000E210E00E9442130091B62A1091B72A36
:104EC0002091252A3091262A021B130B0A551040E7
:104ED0000093B82A1093B92A1091B92A112342F4E9
:104EE000E8EBFAE20081118108591E4F008311831B
:104EF0000E948914E8E2F6E0008100FFFBCF3091C8
:104F0000B92A232F07E010E00E94C80A2091B82A8E
:104F100008E010E00E94C80A20C001E00093C22A05
:104F20000091B42A1091B52A1A930A9325EB34E222
:104F30000FE915E20E94A536229600E80E941803A8
:104F400000E310E00E9442130091CE2A002311F4E6
:104F500001E001C000E00093CD2A08E00E9489032F
:104F600001E00093C22A27EC34E20FE915E20E9427
:104F7000A53600EC0E94180328ED34E20FE915E293
:104F80000E94A53600E80E94180363C60091CF2A4C
:104F900003950093CF2A053018F000E00093CF2A44
:104FA0002091CF2A0EEF11E00E94C80A0091372A03
:104FB0001091382A0E94651002E310E00E9442130B
:104FC00048C6A0E0B0E00E9463138FE591E012C0F4
:104FD000809326099093270904E00E9489030E9488
:104FE000F013A017B1072CF4D8018093232A9093D3
:104FF000242A0496873E03E0900754F30091232A65
:105000001091242A00932609109327090E94201743
:1050100010E400E50E9457133091242A232F01E069
:1050200010E00E94C80A2091232A02E010E00E94AA
:10503000C80A0FC620E035E20FE915E20E94A53646
:1050400000E80E94180300E810E00E94421300E804
:1050500010E00E944213E8E2F6E0008100FDE9C0A2
:1050600000E61AEE0E946510B3950B2FB02F209129
:10507000372A3091382A10E02017310760F701E015
:105080000093C52A2EED34E20FE915E20E94A53601
:1050900000E80E94180300E310E00E94421301E0C0
:1050A0000093C22A02E30E9489032FEE34E20FE943
:1050B00015E20E94A53600E80E94180300E310E004
:1050C0000E94421308E20E94890380E090E0A0E081
:1050D0001EC0E3E5FAE200811181228133810E9442
:1050E0001C30A801B9014A015B01EFE4FAE200813A
:1050F0001181228133810E941C30A401B5010E94DC
:105100007013800F911F08E00E948903A395AA30B5
:1051100000F34AE050E08C010E94532FC801E09157
:10512000B62AF091B72AEA55F040E81BF90BE09354
:10513000B62AF093B72A0091B62A1091B72A0936F9
:1051400021E0120744F0E6EBFAE2008111810856F3
:105150001140008311831091B72A112342F4E6EB2A
:10516000FAE20081118108591E4F008311830E94C9
:1051700071140091372A0E948903E3E5FAE2008165
:105180001181228133810E941C30A801B9014A019A
:105190005B01EFE4FAE200811181228133810E94F8
:1051A0001C30A401B5010E94701348010CEA80165E
:1051B0000FEF90060CF03ECF21E135E20FE915E24A
:1051C0000E94A53600E80E94180305E210E00E9444
:1051D000421305E00E94890305E210E00E94421399
:1051E0000091B62A1091B72A0093B82A1093B92AD1
:1051F0000091B82A1091B92A0E94AE103091B72AB6
:10520000232F05E010E00E94C80A2091B62A06E08C
:1052100010E00E94C80A3091B92A232F07E010E05D
:105220000E94C80A2091B82A08E010E00E94C80A2B
:1052300012CF0091C52A002389F422E235E20FE95A
:1052400015E20E94A53600E80E94180308EE1DEF43
:105250000E94651000E510E00E944213FAC4E8E2E3
:10526000F6E0008100FD37C008EE1DEF0E946510DA
:10527000B3952B2FB22F0091372A1091382A000FA7
:10528000111F30E00217130750F710E400E30E94EB
:10529000571380E090E00AC08C010E947E0A202F04
:1052A0008C0100501E4F0E94C80A0196803002E017
:1052B000900794F324E335E20FE915E20E94A53646
:1052C00000EC0E94180310E200E30E94571308E06C
:1052D0000E94890351CE0091C72A03950093C72AE3
:1052E000033018F000E00093C72A2091C72A08EF86
:1052F00011E00E94C80A08E210E00E94651002E373
:1053000010E00E944213A5C4E8E2F6E0008100FD2F
:105310001AC008EE1DEF0E946510B3950B2FB02F39
:105320002091372A3091382A10E02017310760F792
:1053300000E610E00E9442130E94E91110E200E32F
:105340000E94571319CE0091C12A00950093C12ADB
:1053500002E310E00E94421305E00E94890379C431
:1053600081E090E04091D62A8C010E94292FC8014B
:105370004091D62A0091E42A1091E52A0E94352F07
:105380000170002379F080959095E4EEFAE20081B7
:105390001181082319230083118310E500E40E9482
:1053A00057130CC0E4EEFAE200811181082B192B8F
:1053B0000083118310E300E40E94571301E000937F
:1053C000C42A2091E42A0AE010E00E94C80A309121
:1053D000E52A232F0BE010E00E94C80A3AC401E03E
:1053E0000093C22A08E210E00E94421332C4E8E0AF
:1053F000F6E0008102FD1EC200E00093400900912A
:10540000C92AECE0F4E00C940732E8E0F6E0008111
:1054100002FD25C000E61AEE0E946510B3950B2F21
:10542000B02F2091372A3091382A10E02017310709
:1054300060F70091D42A00950093D42A2091D42AB1
:1054400009EF11E00E94C80A01E00093C52A00E5B7
:1054500010E00E94421301E00E948903FDC3009105
:10546000C52A002381F40091D12A03950093D12A03
:105470000A3018F000E00093D12A2091D12A03E0ED
:1054800010E00E94C80ACEC10091EF2A0395009354
:10549000EF2A013018F000E00093EF2A0E94F9177C
:1054A0002091EF2A0AEF11E00E94C80ABBC10091C7
:1054B000D52A03950093D52A0D3318F001E0009307
:1054C000D52A2091D52A0CEF11E00E94C80A00E4E9
:1054D0001CE90E946510A6C10091DB2A0395009388
:1054E000DB2A093018F008E00093DB2A0BE910E012
:1054F00000932608109327082091DB2A0DEF11E076
:105500000E94C80A8091DB2A90E0019680932A08C5
:1055100090932B0887C18091232A9091242A019788
:105520008093232A9093242A8F3501E0900734F446
:105530000FE511E00093232A1093242A0091232AD7
:105540001091242A00932609109327090E942017FE
:105550003091242A232F01E010E00E94C80A2091F4
:10556000232A02E010E00E94C80A5CC18091B62A9A
:105570009091B72A01968093B62A9093B72A8836DD
:1055800001E0900734F000E010E00093B62A109399
:10559000B72A0E9471140091B62A1091B72A00937D
:1055A000B82A1093B92A3091B72A232F05E010E0CA
:1055B0000E94C80A2091B62A06E010E00E94C80A9C
:1055C00031C18091B82A9091B92A01968093B82A66
:1055D0009093B92A883601E0900734F000E010E09B
:1055E0000093B82A1093B92A0091B82A1091B92AC9
:1055F0000E94AE103091B92A232F07E010E00E94DC
:10560000C80A2091B82A08E010E00E94C80A0AC11E
:105610000091DA2A03950093DA2A093018F008E09D
:105620000093DA2A2091DA2A06EF11E00E94C80AD4
:10563000F9C00091DD2A03950093DD2A053018F0AA
:1056400004E00093DD2A2091DD2A07EF11E00E949B
:10565000C80AE8C00091E12A03950093E12A0330CB
:1056600018F002E00093E12A2091E12A05EF11E011
:105670000E94C80AD7C00091E22A03950093E22A4B
:10568000043018F003E00093E22A0091DF2A0E9420
:10569000E6172091E22A03E110E00E94C80A0E9466
:1056A0002017C0C00091E02A03950093E02A09303A
:1056B00018F008E00093E02A4091E02A50E00FEF54
:1056C00010E00E94212F0E9453112091E02A0CE04B
:1056D00010E00E94C80AA6C00091DF2A039500933B
:1056E000DF2A083018F007E00093DF2A0091DF2A54
:1056F0000E94E6172091DF2A02E110E00E94C80A0A
:1057000091C0E8E0F6E0008101FD1BC000E010E080
:105710000093BC2A1093BD2A0093BA2A1093BB2A87
:1057200004E610E00E94421306E00E94890320E094
:105730000EE010E00E94C80A20E00FE010E00E9496
:10574000C80A0091C12A002309F58091BC2A9091D2
:10575000BD2A01968093BC2A9093BD2A813008E02F
:10576000900734F000E018E00093BC2A1093BD2AA3
:105770003091BD2A232F00E110E00E94C80A209139
:10578000BC2A01E110E00E94C80A20C08091BA2A18
:105790009091BB2A01968093BA2A9093BB2A8836AF
:1057A00001E0900734F000E010E00093BA2A109373
:1057B000BB2A3091BB2A232F0EE010E00E94C80ABA
:1057C0002091BA2A0FE010E00E94C80A2091BC2A5A
:1057D0003091BD2A0091BA2A1091BB2A0E949411DF
:1057E00002E00E9489031EC00091D02A0395009315
:1057F000D02A093018F008E00093D02A2091D02A4E
:1058000004E110E00E94C80A0DC00091D62A039559
:105810000093D62A003118F000E00093D62A01E068
:105820000093C42A08E210E00E94421301E00093B2
:10583000C22A0FC2E8E0F6E0008101FD0AC200E0E2
:10584000009340090091C92AE2E3F4E00C94073286
:10585000E8E0F6E0008101FD2AC000E61AEE0E94B1
:105860006510B3950B2FB02F2091372A3091382A2D
:1058700010E02017310760F70091DC2A03950093B0
:10588000DC2A043018F001E00093DC2A2091DC2AA5
:105890000DE010E00E94C80A01E00093C52A00E56F
:1058A00010E00E94421303E00E948903D5C10091D9
:1058B000C52A002381F40091D22A03950093D22AAD
:1058C0000A3018F000E00093D22A2091D22A04E096
:1058D00010E00E94C80AB6C10091EF2A0A95009311
:1058E000EF2A0F3F19F400E00093EF2A0E94F91706
:1058F0002091EF2A0AEF11E00E94C80AA3C100918B
:10590000D52A0A950093D52A002319F40CE30093B5
:10591000D52A2091D52A0CEF11E00E94C80A00E494
:105920001CE90E9465108EC10091DB2A0A95009344
:10593000DB2A0F3F19F400E00093DB2A2091DB2AD9
:105940000DEF11E00E94C80A8091DB2A90E00196D9
:1059500080932A0890932B0875C18091232A9091F7
:10596000242A01968093232A9093242A883E03E0D8
:10597000900734F007EE13E00093232A1093242AB3
:105980000091232A1091242A0093260910932709B5
:105990000E9420173091242A232F01E010E00E945A
:1059A000C80A2091232A02E010E00E94C80A4AC1D6
:1059B0008091B62A9091B72A01978093B62A909346
:1059C000B72A992332F408E611E00093B62A10931F
:1059D000B72A0E9471140091B62A1091B72A009339
:1059E000B82A1093B92A3091B72A232F05E010E086
:1059F0000E94C80A2091B62A06E010E00E94C80A58
:105A000021C18091B82A9091B92A01978093B82A30
:105A10009093B92A992332F408E611E00093B82A4A
:105A20001093B92A0091B82A1091B92A0E94AE1099
:105A30003091B92A232F07E010E00E94C80A209174
:105A4000B82A08E010E00E94C80AFCC00091DA2AD7
:105A50000A950093DA2A0F3F19F400E00093DA2A3E
:105A60002091DA2A06EF11E00E94C80AEBC00091EB
:105A7000DD2A0A950093DD2A013018F401E0009335
:105A8000DD2A2091DD2A07EF11E00E94C80ADAC062
:105A90000091E12A0A950093E12A013018F401E00F
:105AA0000093E12A2091E12A05EF11E00E94C80A43
:105AB000C9C00091E22A0A950093E22A013018F445
:105AC00001E00093E22A0091DF2A0E94E61720916C
:105AD000E22A03E110E00E94C80A0E942017B2C027
:105AE0000091E02A0A950093E02A0F3F19F400E0A4
:105AF0000093E02A4091E02A50E00FEF10E00E946E
:105B0000212F0E9453112091E02A0CE010E00E9406
:105B1000C80A98C00091DF2A0A950093DF2A013055
:105B200018F401E00093DF2A0091DF2A0E94E617B3
:105B30002091DF2A02E110E00E94C80A83C0E8E059
:105B4000F6E0008102FD11C000E010E00093BC2AE5
:105B50001093BD2A0093BA2A1093BB2A04E610E0E2
:105B60000E94421306E00E9489030091C12A00238B
:105B7000F9F48091BC2A9091BD2A01978093BC2AA8
:105B80009093BD2A992332F400E010E00093BC2AE0
:105B90001093BD2A3091BD2A232F00E110E00E940E
:105BA000C80A2091BC2A01E110E00E94C80A1EC068
:105BB0008091BA2A9091BB2A01978093BA2A909338
:105BC000BB2A992332F407E611E00093BA2A109316
:105BD000BB2A3091BB2A232F0EE010E00E94C80A96
:105BE0002091BA2A0FE010E00E94C80A2091BC2A36
:105BF0003091BD2A0091BA2A1091BB2A0E949411BB
:105C000002E00E9489031EC00091D02A0A950093E9
:105C1000D02A0F3F19F400E00093D02A2091D02A17
:105C200004E110E00E94C80A0DC00091D62A0A952E
:105C30000093D62A0F3F19F40FE00093D62A01E013
:105C40000093C42A08E210E00E94421301E000938E
:105C5000C22A00E00093C52A0091D42A002349F00B
:105C6000009164060F73009364060AE20093B32A5E
:105C700008C000916406006C0093640600E2009383
:105C8000B32A8091480690E08C7090700091F02AC1
:105C900010E00817190711F40C947B1C8093F02A6C
:105CA0000091F02A0C3029F401E00093EE2A0C94C4
:105CB0007A1C0091F02A083011F00C94731C00E05B
:105CC0000093EE2A0C947A1C00008895FECF0E9467
:105CD0005432C801D9012A013B015CD057D071F47C
:105CE0008201930153D051F401E2E7EFFAE200831D
:105CF00041830FEF1FEF2FE73FE73DC044D0A201E4
:105D0000B3010E947B30AC01BD0140D061F442D0B0
:105D10003AD00E94F6310BED1FE029EC10F43FE37E
:105D20002AC03FEB28C0A201B3012DD00E945531FB
:105D3000080119012FD0820193010E94DE3123D086
:105D4000A0F41CD050F424D0A801B9010BED1FE041
:105D500029E430E40E94BF300EC01AD04BED5FE062
:105D600069E470EC0E947B3006C008D010F410D0BB
:105D700002C00ED03058E8E00C9465320E94F63133
:105D80008001910108958C019D0108950C94D431F6
:105D90000C94563540E050E060E070E008953F77A5
:105DA00041E00C94F53503E20DBF01E20EBFC0E007
:105DB000D1E20E94F532002311F00E94D8350E94F2
:105DC00080180E94642E0C94642E0D01DA0140E0CC
:105DD00050E060E070E00E94D43139F400E010E05F
:105DE0004D934C9320E030E00CC0B901660F771F53
:105DF0007E57572F550F550B7D935C932F77307837
:105E00003F63D00108950024E8E0EA9532F0001FD6
:105E1000001C0416D0F3041AF8CF001F402D009583
:105E20000895FF27442312F4F1604195002312F4F2
:105E3000F09501950E94032FF0FD0195F1FD41952C
:105E40000895149F102D059F100D049F002D110D16
:105E500008954A951AF0000F111FFBCF08954A9537
:105E60001AF016950795FBCF08954A951AF01595E7
:105E70000795FBCF089500241124EFE0001F111FA8
:105E8000001C111C0416150610F0041A150AEA95D8
:105E9000AAF7001F111FA0010095109508955195B4
:105EA000419550400895FF27552312F4F160F7DF24
:105EB000112312F4F09507D00E943B2FF0FD03D080
:105EC000F1FDEDCF0895119501951040089522241C
:105ED000349F302D259F300D169F300D079F300DBC
:105EE000249F202D310D159F200D311D069F200D63
:105EF000311D149F102D210D321D059F100D211DE8
:105F0000321D049F002D110D221D321D08954A954A
:105F10002AF03695279517950795F9CF08954A9554
:105F20002AF03595279517950795F9CF0895002400
:105F300011241001E0E2EA9592F0001F111F221FC8
:105F4000331F001C111C221C331C041615062606C8
:105F5000370688F3041A150A260A370AECCF001F01
:105F6000111F221F331FA001B1010095109520952C
:105F700030950895FF27772312F4F16015D033236D
:105F800012F4F09509D00E94972FF69508F404D0EA
:105F9000F69508F409C0089530952095109501955F
:105FA0001F4F2F4F3F4F0895709560955095419525
:105FB0005F4F6F4F7F4F0895FF27112477FB660FC8
:105FC000771F089409F4771F679517F8EE270024C8
:105FD00037FB220F331F089409F4331F279507F866
:105FE000089527FD0EC0EE0F001F111F221F3A95C6
:105FF0003230B8F7332319F427FD31E002C027FF10
:1060000030E0E03821F400FF08940EF488940F4F3C
:106010001F4F2F4F3F4F323038F4332319F427FDF1
:1060200031E002C027FF30E03F3F29F0220F000C93
:10603000379527950895ACC0032E002012F40E94D6
:10604000CC2FE02F012F122F232F3EE9D1CF002498
:10605000F8CFBCDF432F4F5748F04F3148F007FCD3
:1060600091C03FE72FEF1FEF0FEF089533278CC04C
:10607000322F212F102F0E2F4F5141950E94872F25
:1060800007FE08950C94CC2FF901EE0FFF1F37FB8C
:10609000FF3F31F0EF2BE12BE02B8894B89408956B
:1060A000E02BE12B21F008949894B89408959894EB
:1060B000889438940895FB01EE0FFF1F77FBFF3F94
:1060C00031F0EF2BE52BE42B8894B8940895E42B62
:1060D000E52B69F3E8CFEFDF68F021F43723262FB3
:1060E0008A010895372FFBCFE6DF20F00BF00895EB
:1060F0007327EAF751C0C8DFE8F3B3F361F3DBDFDE
:10610000C8F383F3A1F358DF401751076207730701
:1061100031F4011411F10024E89488942BC078F034
:10612000332E372F732D322E262F632D312E152F20
:10613000532D302E042F432D302C012C132C3717C8
:1061400039F0669557954795F795E0407395F7CFE9
:10615000E7FBEE0FE0E010246AF0EF0F041F151FBD
:10616000261F60F4279517950795E79508F468941E
:1061700033953ECFEF0B040B150B260B39CFE0E820
:106180007E27B9CF302D3078222711270027089598
:106190003FE7302920E8F9CF3FEF2FEFF6CF8BDF35
:1061A000D8F3D1F370783727089585DFA8F3A3F3E8
:1061B000F9CF3078372793CF67DF70F383F3A9F3F4
:1061C0007ADF50F3B3F3A9F3F7DE0124E8943F57E5
:1061D000E040370FEF1F12F0D9F603C03A3E90F2BD
:1061E0006894E0E00A92AA933A93AA2733242224DF
:1061F0003327049FF001059FF00D712D731F149F2D
:10620000F00D711D221C069F700D211C331C159F63
:10621000700D211C331E249F700D211C331E169FF0
:10622000200C311CAA1F259F200C311CA31F269F68
:10623000300CA11D39915EF43395A69537942794BF
:106240007795F795E79533953130BCF316C0AA23BF
:1062500022F0332351F4339510C0339571F4A99192
:10626000099096CFA7FD09C03A95EE0FFF1F771F43
:10627000221C331CAA1F3230A8F7E894FE2B09F029
:1062800068942A2F8101E72FA9910990BACE13DFD4
:1062900010F00BF087CF80CF0EDFE9F3E0F3032E91
:1062A000072670CF032E072673CFEEDEA0F37BF315
:1062B00099F301DF80F39BF3A9F37EDE012427FD30
:1062C00006C0000F111F221F3150E040F8CF67FDBC
:1062D00006C0440F551F661F7150F040F8CFE89478
:1062E000371BEF0B3158EF4F2AF0EE23E9F63F3F13
:1062F000D9F203C03A3EA8F26894E0E0F0E011243D
:10630000139440175107620738F0315008F468942D
:10631000000F111F221FEE1F041B150B260BEF0B86
:10632000000F111F221FEE1F0A9279E17A95AAF041
:10633000041715072607EF0730F0041B150B260B73
:10634000EF0B089401C08894111C221C331C001C04
:10635000000F111F221FEE1FE9CFF0F9E894E22B86
:10636000E12BE02B09F06894069437942794179456
:10637000E79508F468947395B9F30990332311F005
:10638000F0FF09C0369427941794E79508F46894B1
:1063900033953130BCF3012D122D232D32CE8BCE0F
:1063A00098940895189408956FDED0F3C1F383DEB6
:1063B000B8F3041715072607370708957CDEA0F009
:1063C00063DE90F029F0E32FE7273AF4731708957E
:1063D00072DE51F04EF00894089504171507260751
:1063E000370719F016F4B8F78894089564DEE0F3DF
:1063F0004BDED0F3E7DFC0F3089408957591659103
:1064000055914591159011FA259035900895F9DF31
:10641000041B10E003C0F4DF041B150B20E030E088
:1064200005C0ECDF041B150B260B370BB8F010FC76
:1064300017C045910590E00FF11F0417100540E0CB
:106440002407340758F436F404910024F101E01BCA
:10645000F0090994E00FF11F25903590F10109949E
:1064600011F4D6F7F1CF31960EF0319650E060E09E
:1064700070E045914B3F48F089F34F3F29F04E3F84
:1064800011F07591659155914591041B150B260BE3
:10649000370B39F318F3E7CFFA92EA92DA92CA92FD
:1064A000BA92AA929A928A927A926A925A924A924C
:1064B000BA93AA939A938A930895FF84EE84DD8415
:1064C000CC84BB84AA84998488847F806E805D801C
:1064D0004C80BB81AA8199818881F0E0EC0FFD1F7F
:1064E000EF0108950E945032229741E050E060E0B1
:1064F00070E00E94DE3160F440E00E94D43121F46B
:1065000002E26BD03FEF5FC001E267D03FE75BC0C4
:10651000AE010E94E52EC801D90143EF54E065E3C6
:106520007FE30E94DE3168F437FBAA0FBB1FB395EF
:10653000B695A795B7F908811981015010400883D5
:10654000198340E050E060E87FEB43D02801390137
:1065500040E050E060E87FE33CD0A801B90182014F
:1065600093010E945531C801D901A801B9012FD06A
:10657000280139010881102F110F110B212F312F04
:106580000E941C3048E152E761E37FE320D04801DC
:10659000590142E252E964ED7EE38201930117D092
:1065A0004DED5BE96AE27FE316D0A201B3010FD0A3
:1065B00044E050E060E070E40ED0AC01BD0107D0D3
:1065C000A401B50108D02296ECE00C9461320C9441
:1065D000DC308C019D010C947B30E7EFFAE2008304
:1065E00051830FEF1FEF2FE7089501E008950E94F8
:1065F0004C32EF97EF976A972A873B8748875987EE
:1066000068017B0100E00B830C8302C011D21BD216
:106610000AD2053251F00023C9F70B811C81EF9695
:10662000EF966A96E0E10C945D320081053221F428
:1066300002D2FED105E2EBCF00E00F830E830A8386
:1066400009833E0102E1600E00E0701E07E415E2DE
:10665000088B198B06C00981002311F4008109837E
:10666000EAD1D9D10052B9F3035059F00850B1F32F
:10667000025019F0035049F00CC00A8103950A83B7
:10668000EFCF0E8103950E83EBCF0F8103950F8320
:10669000E7CF00810A3279F4AAD1AD90BD9098D1AC
:1066A000BB203AF4B194A19400E0B00A0A810395AA
:1066B0000A83C1D114C0AA24BB244AE050E00DC013
:1066C00021916F0185010E94212FA22EBB24A00ED3
:1066D000B11E00EDA00E0FEFB01EA0D188F30A810D
:1066E000002311F000E00F8396D10E32F1F4A3D114
:1066F00092D10A3231F47BD18D909D9069D19BD19A
:1067000017C0882499244AE050E088D188F4219168
:106710006F0184010E94212F822E9924800E911EE8
:1067200000ED800E0FEF901EF0CF88248A94982CF5
:1067300080E071D10C5421F00C5131F0045039F447
:1067400081E0C80E7AD103C001E0C00ED81E6BD123
:10675000E8E5F4E00C94073280FB5EF44B815C8149
:10676000652F660F660B47D1408351836283638335
:106770004FCF2B813C813FD12083318349CF37D10B
:106780000D91119625D10A8B2E0103E115D1E0C0A0
:106790002ED16D907D901CD1062D072921F408E59E
:1067A000602E05E2702E992022F400E1802E07E28F
:1067B000902E80E090E001C00196F30101913F012D
:1067C000002319F088159905BCF30CD1230191958C
:1067D00081959040680E791EBBC00E81002331F078
:1067E000082D092919F499248824839407E615E2D1
:1067F000088B198B0881003739F4F9D0ECD000E10F
:10680000D5D000E0098330C0F1D046F40D911D9140
:106810002D913D91DDD0C801D90101C0DCD00881A6
:106820000F3611F408E0ECCF053749F70AE0E8CF5E
:10683000DDD04D915D9126F46D917D91C9D005C05B
:10684000C7D0652F660F660B762FCA01DB01772351
:106850004AF40DE209839095A095B09581959F4FDC
:10686000AF4FBF4F0AE0A2D03E0107E9600E00E043
:10687000701E2E0107E9A0D0082F092B0A2B0B2B25
:1068800011F001E001C000E00D83082D092919F481
:106890000D8100FF1FC094D0E889F989E00DF11D3A
:1068A0000081F30102933F018BD0C801D901012B74
:1068B000022B032B81F799206AF40F81002351F0FA
:1068C000A3D010E04501801A910A04C000E3F3014F
:1068D00002933F018E0109561F4F0619170908152B
:1068E0001905A4F30E81002399F10D8100FF30C03A
:1068F0000881083711F0083549F474D0F301088194
:10690000008370D000E3F301008322C00F3601F54D
:10691000F30100810033E1F000E302933F0118C06E
:1069200008E7602E05E2702E462C502EF201008101
:10693000002371F001E040D0F9CF0FEFC00ED01E60
:106940000BE9602E05E2702E0EE9402E05E2502E76
:10695000420186189708A814B9041CF480E090E05E
:1069600007C052D0A818B90810E0A01AB10AC50192
:106970000A81002321F401C063D00197EAF709815D
:10698000002339F055D004C053D0F30101913F01E9
:106990005AD00FEF800E901EBAF70A81002309F437
:1069A00037CE01970AF434CE4BD0FBCF10E00C87E2
:1069B0001D871E871F870895400E00E0501E089512
:1069C0004C855D856E857F858C019D010C94972F8C
:1069D000A083B18308958D919D91A083B183A0E0A0
:1069E000B0E008950FEF600E701E089580FBF70170
:1069F000A081B1810895F701A081B1810D911D9110
:106A0000A083B183F80108950981002311F001E00A
:106A1000089500E00895F60100810895F6010081CF
:106A200000530A300895F60101916F01088308951B
:106A300028853985089501E0C00E00E0D01E089534
:106A40002885398500E2EA85FB8509950B811C8143
:106A50000F5F1F4F0B831C8308950E945832C8019B
:106A6000D9011A013F7740E856E968E17BE40E94CA
:106A7000F63138F416D0B38300E010E020E030E0C7
:106A80000DC03B2F0E9429300E941C300AD0338356
:106A9000A801B9018C019D010E94BF30E4E00C9473
:106AA0006932F10100831183228308950E944C32E0
:106AB000C801D901BF7741E050E060E87FE33B2F98
:106AC0000E94DE3170F440E00E94D43129F40BEDD5
:106AD0001FE029E43FE350C0CC24DD24EE24FF2452
:106AE0001CC00BEDC02E0FE0D02E09E4E02EF72ED7
:106AF00040E07FEB082F48D02801390140E050E00A
:106B000060E87FE38C019D013FD0A801B9018201BB
:106B100093010E945531C801D901AC01BD018C011E
:106B20009D012DD02801390144E25FEF6BE27CEB3F
:106B300026D048E854E466EA7EE328D048E150ECE9
:106B40006FE370E423D045EB1CD0480159014AEEB5
:106B500054EB66E870E48201930118D046EB11D043
:106B6000A801B901840195010E945531AC01BD0114
:106B700006D0A601B70108D0E0E10C945D320C9478
:106B8000DC305DEF68E670E40C947B30FDDFA20141
:106B9000B301F5CF20E006D0E9F70895259102D0A2
:106BA000E9F708952D9301501040202F212B0895CF
:106BB0008AE69EE6FC0105911491FC013296A591AE
:106BC000B491FC01349625913491422F432B19F056
:106BD000F901E4DF01C0DEDF06961EE68637910785
:106BE00048F3089540E00C94F5350E9454322897FC
:106BF000802FB32F442E40E050E060E070E00E9410
:106C0000DE3110F401E001C000E0000F400EBF775C
:106C100043E859EF62E27FE3082F3B2F80D076D024
:106C200041E05CEF6FE777E40E94F63188F5AE0152
:106C30000E942D356BD0042D10E06BD04881598116
:106C40006A817B8172D0088319832A833B83AE01DA
:106C50004C5F5F4F2A0140E050E060E87EE35FD088
:106C6000A2010E942D3540E050E060E870E40C8104
:106C70001D812E813F8153D0A801B901088119815E
:106C80002A813B810E94BF300E942930402E0CC0D7
:106C90000E942930602E3DD0A801B9018C019D01D0
:106CA00033D0460C03E0402240FA3EF4AC01BD0173
:106CB00000E010E020E83FE327D002E0401608F0B3
:106CC000B0588C019D0129D0280139014BEF57EDB7
:106CD0006EE179E324D045E656E269E97BEB21D009
:106CE00048E554E363EA7DE31CD041EE5DE565E2EF
:106CF0007FEB17D04BED5FE069EC7FE316D00DD052
:106D00002896E8E00C9465320E94BF30C801D90192
:106D1000089520E030E00C942730AC01BD010C94C4
:106D2000DC3003D0A201B301FACF0C947B301B2FCF
:106D30006A2FF901A081B181AD014F5F5F4F4083A0
:106D400051830C93A62FB12F0895BA93AA93249739
:106D50000A831B8389019E012A5F3F4F2883398361
:106D6000BE01AE014E5F5F4F27E936E30E94F73266
:106D700020E0AA81BB812C932496A991B991089512
:106D80000E94503222974801590141E050E060E0F2
:106D900070E00E94DE3198F440E00E94D43129F482
:106DA00000E010E020E030E04EC001E2E7EFFAE260
:106DB000008351830FEF1FEF2FE73FE744C0AE0181
:106DC0000E94E52EC801D90145EC53E062E47FE35F
:106DD0000E947B304AE151E562E17FE33BD0A801AC
:106DE000B9018C019D013BD0402E088100FF14C0E9
:106DF0000A952DD0802F43EF54E065EB7FE3042DFF
:106E00000E94DC3037FB220F331F380F3695279551
:106E100037F9C801D9010BC01AD0842D912FD9019F
:106E200037FBAA0FBB1FB00FB695A795B7F940E087
:106E300050E060E87EE38C019D010CD0AC01BD0107
:106E4000840195010CD02296ECE00C94613242E072
:106E50000C94112F0E94DC302801390108950E9402
:106E60005531A201B3010C947B307B042421766E52
:106E70005A059F2500004E6F726D61005475726255
:106E80006F00547265736800547572626F31004F01
:106E90006666004F6E00496E760076646920005683
:106EA00044492000537664690053564449002D201C
:106EB000504C454153452057414954202D20002036
:106EC0002020202020203C3E2020202020202000A8
:106ED000204C6F77204261747465727920212121E2
:106EE000002020203C20256420487A203E202020BD
:106EF00020002045524153494E4720454550524FAE
:106F00004D212000726164696F646F6D2E75636F2F
:106F10007A2E7275004B504F54332D34382D474123
:106F2000494E2D53256300466163746F7279207357
:106F3000657474696E6773002020205365747469EA
:106F40006E6773202020202000553D256420493D98
:106F5000256420456D3D2564202020004D3D25649D
:106F600020413D25642047623D256420473D25643E
:106F700020005458202564487A2025646D41202043
:106F80000052582025646D562020202000473D25C2
:106F9000642A257320002020205475726E20636FB0
:106FA000696C2120202000436F696C20626C3F20B7
:106FB00059657320272B2700202020202020202007
:106FC0002000202564256446256425630025647619
:106FD000256420002B253032645B002D253032647F
:106FE0005B005D20532564256446256425630025E8
:106FF000647625640020202020202F2020202020BF
:107000002020202020002020202020202050502040
:107010002020202020200025642020202020200067
:1070200050726F66696C652020202020202020206F
:10703000200054623D25642E256456202055623D73
:1070400025642E256456200042617474657279208F
:10705000202020203C25643E002B25642020202079
:107060002D2E2E2E2E2E2E2E2E2B00436F6E747252
:107070002E20202020202020202020200025646D8C
:1070800041202020202020202020202020202000FF
:10709000282564292E2E2E20002A467265715F5401
:1070A0005820256C64487A20002A466572726974FB
:1070B0006520200020202564256320200047726F72
:1070C000756E6420626C2E2000534C2E25732000B8
:1070D0002D2E2E2E2E2E2E2E2E2B00566F6C756DD5
:1070E000652020202020202020202000506F6C7957
:1070F0007068002564746F6E65200042656570736A
:107100002020202020202020202020002573202047
:107110002D2E2E2E2E2E2E2E2E2B00496E646963C0
:107120002E20202020202020202020200025732019
:107130002D2E2E2E2E2E2E2E2E2B004D6F646520E2
:107140002020202020202020202020200025646DC9
:107150004120202000506F7765722E2020202020B3
:107160002020202020002A256420202020004761A4
:10717000696E202020202020202020202020002593
:10718000646D562020202020200020413D256420D1
:107190002020002A436F696C20626C2E20663D25FA
:1071A00064256320200025642020202020004850F2
:1071B00046202020202020202020202020200038B1
:1071C000363432302F30313233343536373853009D
:1071D0002020202825303264293C253032643E208E
:1071E000202020200047726F756E6420626C2E454F
:1071F00072726F72210047726F756E6420626C2E1E
:10720000202D4F4B2D20002020202A2A2A202564C3
:10721000202A2A2A20202020002020202020202070
:10722000202020202020202020002B30305B200038
:1072300020204E6F204665727269746521202020DF
:10724000002054616B652046657272697465212067
:10725000200020202020204572726F7221202020E3
:107260002020002020202020204F4B2120202020E3
:10727000202020002020202020206C6F6E672020FE
:107280002020202020002A2A205752414954204FF4
:107290004B21202A2A2000900130313233343536F8
:1072A00037383941424344454600286E756C6C209E
:1072B000706F696E7465722900303132333435363F
:1072C00037383961626364656600464C4F415453F8
:1072D0003F2077726F6E6720666F726D61747465A0
:1072E0007220696E7374616C6C656421003F3F3F6E
:0172F000009D
:0400000300000000F9
:00000001FF
